:020000040800F2
:10000000C81D00200101000821550008DD3D000841
:1000100065530008C10F000851810008000000006E
:10002000000000000000000000000000DD65000886
:10003000B72D000800000000C95A00080569000833
:100040001B010008855800081B0100081B0100085F
:100050001B0100081B0100081B0100081B01000810
:100060001B0100081B0100081B0100081B01000800
:100070001B0100081B010008DD2800081B01000807
:100080001B0100081B01000859070008297C000813
:10009000D57C00081B010008E90F00081B010008BF
:1000A00095690008916A00081B0100081B010008FF
:1000B000956A00087D6D0008D96F00081B010008D3
:1000C0001B0100081B0100081B0100081B010008A0
:1000D0001B010008797B00081B0100081B010008B8
:1000E0001B0100081B0100081B010008DFF80CD0F1
:1000F00000F0F4FA0048004765970008C81D00208A
:100100000648804706480047FEE7FEE7FEE7FEE7B1
:10011000FEE7FEE7FEE7FEE7FEE7FEE721690008EF
:10012000ED0000082DE9F0410024061B254671F181
:10013000000605DA01240027D0EB070067EB010178
:10014000161E73F1000605DA0027D2EB070201251F
:1001500067EB030300F0DEF986460E4617469C4621
:10016000AC4204D00025D0EB050E65EB010624B1AE
:100170000020D2EB000760EB030C704631463A4694
:100180006346BDE8F08140EA01039B0703D009E024
:1001900008C9121F08C0042AFAD203E011F8013B73
:1001A00000F8013B521EF9D2704710B5002200E062
:1001B000521C835C8C5CA34201D1002BF8D1D8B2D5
:1001C000E1B2401A10BD80EA010210B502F000430E
:1001D000400022D04A001FD0010E01EB1261C0F393
:1001E0005600C2F3560240F4000042F40002A0FBA5
:1001F000022000047F39140400D0401C50EA124051
:1002000001D44000491EC2B20C0604EBD010401CC1
:100210004008802A02D003E0002010BD20F0010039
:10022000002900DA0020184310BD2DE9FE4F81EAB5
:10023000030404F0004421F0004100944FF0000B4F
:1002400023F0004350EA01045ED052EA03045BD07D
:10025000C3F30A54C1F30A552C44A4F2F3340194B5
:10026000A0FB0254C1F3130141F48011C3F3130343
:1002700043F4801301FB024400FB034E840A970AF7
:1002800044EA815447EA8357A4FB076802958D0A24
:1002900005FB07854FEA932C04FB0C542705029DB0
:1002A0004FEA065847EA1637B5EB08056EEB070C20
:1002B000870E920E47EA811742EA8312A7FB0201DA
:1002C000B6EB0B0164EB00042B0D43EA0C335E1814
:1002D00044EB1C50DA465146E7FB0201C5F3130418
:1002E0004FEA0B3343EA14534FEA0432019C43EACA
:1002F0000603A4F10C040294009CCDE900B400F0C4
:100300009FF903B0BDE8F08F00200146F9E72DE921
:10031000F04D81EA030404F0004B21F0004514463F
:100320004FF0000A23F0004150EA050220D054EAC1
:1003300001021DD0C5F30A570246C5F31303C1F3EA
:100340001300C1F30A5640F4801543F48013A7EB61
:100350000608101BD64608F2FD3873EB050002D3E1
:1003600008F1010801E092185B41B8F1000F03DACF
:1003700000200146BDE8F08D00204FF480110646B4
:1003800084460EE0171B73EB050705D3121B63EBC6
:10039000050306434CEA010C49084FEA3000921865
:1003A0005B4150EA0107EDD152EA030012D082EA24
:1003B000040083EA0501084305D0101BAB4106D2B7
:1003C0000122002306E000224FF0004302E06FF01C
:1003D000010253101AEB06004CEB085110EB0A0017
:1003E00041EB0B01BDE8F04D00F01BB970B521F0F9
:1003F000004303430CD0C1F30A550024D5EB040598
:1004000064EB0403D617AD1AB34102DB00200146AA
:1004100070BD201841EB025170BDC10F80EAE07041
:100420000844CA079623002100F0CDB89623002285
:10043000114600F0C8B80EB5C10F80EAE07008445C
:10044000CA07002140F233438DE80E000A460B46EE
:1004500000F0F6F803B000BD0EB540F23341029152
:100460000021CDE900110A460B4600F0E9F803B07F
:1004700000BD00F0004220F00040C10DC0F31600A6
:1004800040F400007F2901DA00207047962903DC40
:10049000C1F19601C84001E096398840002AF4D0A5
:1004A0004042704770B5C1F30A5201F00045002484
:1004B000C1F3130140F2FF3341F480119A4201DA93
:1004C000002070BD40F233439A42A2F2334203DC73
:1004D000524200F05FF800E090402C43F1D04042DF
:1004E00070BDC1F30A5210B5C1F3130140F2FF33DE
:1004F00041F480119A4201DA002010BD40F23343EA
:100500009A42A2F2334203DC524200F043F810BD9B
:10051000904010BD2DE9F05F0546002092469B46B5
:1005200088460646814640241BE028464146474609
:10053000224600F02FF853465A46C01A914110D374
:1005400011461846224600F016F82D1A67EB0108EE
:100550004F4622460120002100F00DF817EB00095C
:100560004E41201EA4F10104DFDC484631462A46F4
:100570004346BDE8F09F202A04DB203A00FA02F14E
:10058000002070479140C2F1200320FA03F3194381
:1005900090407047202A04DB203A21FA02F0002123
:1005A000704721FA02F3D040C2F120029140084383
:1005B000194670470029A8BF7047401C490008BF72
:1005C00020F00100704710B4B0FA80FC00FA0CF083
:1005D00050EA010404BF10BC704749B1CCF12004BB
:1005E00021FA04F411FA0CF118BF01212143084348
:1005F000A3EB0C01CB1D4FEA00614FEA102042BF74
:10060000002010BC704700EBC35010440029A4BF69
:1006100010BC7047401C490008BF20F0010010BC0E
:10062000704710B5141E73F1000408DA401C41F144
:10063000000192185B411A4301D120F0010010BD66
:100640002DE9F04D92469B4611B1B1FA81F202E0DC
:10065000B0FA80F220329046FFF78DFF04460F4635
:1006600040EA0A0041EA0B0153465A46084313D0B8
:10067000114653EA010019D0C8F140025046FFF775
:1006800089FF05460E46504659464246FFF773FF1E
:10069000084305D0012004E020463946BDE8F08D2E
:1006A0000020054346EAE0762C4337430A98630569
:1006B000E40AA0EB08000022FD0A44EA47540A308D
:1006C00002D500200146E9E7010510196941DDE97D
:1006D000084500196941BDE8F04DA2E7064C074DF9
:1006E00006E0E06840F0010394E807009847103402
:1006F000AC42F6D3FFF7FEFC48B9000868B9000821
:1007000070B58C1810F8015B15F0070301D110F8D3
:10071000013B2A1106D110F8012B03E010F8016B00
:1007200001F8016B5B1EF9D12B0705D40023521E83
:100730000DD401F8013BFAE710F8013BCB1A921CEB
:1007400003E013F8015B01F8015B521EF9D5A142E9
:10075000D8D3002070BD000070B54A4C4FF49065AE
:100760002946204600F017FA002860D02946204686
:1007700000F09EF844490888401C0880012120466A
:1007800000F0E8FA414942F21072B1F85800904284
:1007900002D2401CA1F8580009F01AFA3C4DB5F9F4
:1007A0001410B5F9120007F0C1FE3A4CA5F8560036
:1007B0002080A16820468847A088A5F8580004F04A
:1007C00019FF09F005FB344E344C307808282FD03F
:1007D00045F6AC30606042F6EF60A06042F2C400C3
:1007E000E0602F48008A2080208E6080A16B2B481B
:1007F0008847208E40F21C7180002A4C00EB81005B
:100800006887A2684FF0000550071AD5264840F2C5
:100810001A63C188491C89B2C180994207D3234B0E
:1008200049F68141198022F00401A160C58070BDA4
:1008300041F2130060604FF48060A06040F61B50EE
:10084000CEE730780A2818D2DFE800F01706130543
:100850000A050D171113EAE7BDE8704008F03CB82F
:100860000AF058FA05E0BDE8704004F04FB808F00F
:100870004FFDBDE8704009F003BC01F0F1FD84F8C4
:10088000BA5070BD00240140480700203801002004
:100890004C000020300700203F070020CC00002043
:1008A000F0010020A4020020C80A0020442C0140CE
:1008B0006FEA1121016070470029816802D041F080
:1008C000010101E021F00101816070470029816888
:1008D00002D041F4807101E021F4807181607047A1
:1008E0002DE9F041854E92B0304600F011F90BA889
:1008F00000F03FFA01214FF4C06005F079F90024BF
:100900008DF831404FF46020CDE90D044FF4A02064
:100910004FF00A080B9001278DF83C808DF830705D
:100920000BA9304600F086F9754D8DF831408DF8F1
:1009300030708DF83C700BA9284600F07BF901233C
:100940001A460F21304600F0C6F902220123114653
:10095000304600F0C0F9012303221946304600F06A
:10096000BAF9012304220021304600F0B4F9012332
:1009700005220321304600F0AEF9012306220821AA
:10098000304600F0A8F9012307220A21304600F082
:10099000A2F9012308220B21304600F09CF9012323
:1009A00009220D21304600F096F901230A22042184
:1009B000304600F090F90121304600F084F9012121
:1009C000284600F080F901231A460521304600F040
:1009D00055F901231A460621284600F04FF9002157
:1009E000304600F0CBF84FF4E041284600F0C6F85E
:1009F0000121304600F0B8F80121284600F0B4F893
:100A00000121304600F0A6F80121284600F0A2F8A6
:100A10000121304600F09EF90121284600F09AF9A4
:100A200040F61451374806F0AEFD12208DF8400014
:100A300002208DF841008DF842408DF8437010A8D7
:100A400004F09CFD01224FF49061304600F0E8F87C
:100A500001213046FFF73AFF01213046FFF72CFF16
:100A600001212846FFF728FF304600F06EF9304696
:100A700000F09FF80028FAD1304600F075F93046B2
:100A800000F082F80028FAD1284600F05EF92846E6
:100A900000F08FF80028FAD1284600F065F92846C2
:100AA00000F072F80028FAD10121084605F07CF820
:100AB000154D284601F04EFF684601F0EEFF0F4845
:100AC00001A94C300090114881E811018020CDE946
:100AD00004404000069080000790202008904FF4CA
:100AE0004050CDE909046946284601F0B9FF0121CB
:100AF000284601F023FF12B0BDE8F0810024014038
:100B000000280140002C014008000240B4020020EF
:100B10000D4910B5884202D1012144150AE00B4964
:100B2000884202D10121041504E0094988420AD112
:100B30000121CC03204605F067F82046BDE81040AF
:100B4000002105F061B810BD0024014000280140DB
:100B5000003C01400029816802D041F4801101E08D
:100B600021F48011816070470029816802D041F42E
:100B7000004101E021F4004181607047826822F465
:100B8000E0420A43826070470146002089684907B5
:100B900000D50120704710B50246002054680B0AAA
:100BA000C9B20C401168194202D0002C00D00120BB
:100BB00010BD014600208968090700D50120704753
:100BC00038B501211C2005F013F8EF20ADF8000026
:100BD00000248DF8034003258DF8025069460D4826
:100BE00002F006FD0120ADF800008DF803408DF8FD
:100BF00002506946084802F0FBFC3B20ADF80000BB
:100C00008DF803408DF802506946044802F0F0FC6C
:100C100038BD000000080140000C014000100140F8
:100C2000002A4268C9B201D00A4300E08A43426008
:100C30007047000010B542680E4B0C791A400B68E3
:100C400042EA04221343436083680B4A1340D1E90C
:100C5000024222434C7943EA44031A438260C26A47
:100C6000097C22F47002491EC9B242EA0151C162F4
:100C700010BD0000FFFEF0FFFDF7F1FF70B5072487
:100C800009290AD9C568A1F10A0606EB4606B4404F
:100C9000A543B3401D43C56007E0056901EB41066C
:100CA000B440A543B3401D430561836BC3F30154B6
:100CB000121B921C02EB82041F22A2409343A1400C
:100CC0000B43836370BD826B491E22F4401242EADB
:100CD00001518163704770B5072409290AD9C56895
:100CE000A1F10A0606EB4606B440A543B3401D43F6
:100CF000C56007E0056901EB4106B440A543B34078
:100D00001D4305611F23072A09D2446B521E02EBC3
:100D1000820293409C4391400C43446370BD0D2A72
:100D200009D2046BD21F02EB820293409C43914094
:100D30000C43046370BDC46A0D3A02EB8202934017
:100D40009C4391400C43C46270BD816841F008012E
:100D5000816070470029816802D041F4A00101E060
:100D600021F4A00181607047816841F00401816035
:100D7000704700210160017141718160C1600121F2
:100D800001747047002800DA4042B0F5803F02DB72
:100D90004FF6FF70704780B27047000070B51E4C70
:100DA000214694F83800B1F8425006281ED9B4F80C
:100DB0004A10B4F84C00A1EB000202F10902122A19
:100DC00004D8FFF749FB0022144B0AE0884204D202
:100DD000FFF742FB0022124B03E0FFF73DFB00222E
:100DE000104BFFF722FAFFF77CFB09E005D12846FC
:100DF000FFF732FB0C4A0D4BF3E70D4951F8200089
:100E0000C5EB45116063B0EB410F03D9C5EB45104D
:100E10004000606370BD00005804002000003440B2
:100E200000003340000035406766666666E64B406A
:100E3000CCAF000810B50C4C2078400713D5FFF755
:100E4000ADFF0A49A08E088008483038018821F09B
:100E500010010180001F018841F0100101802078FD
:100E600020F00400207010BD580400204004004011
:100E7000F0B4254B002103F134009A793AB1234AAA
:100E800041F2CD05B2F90240AC4211DC99711E4C21
:100E900082683434C2F3C006C2F300252468AE422F
:100EA00011D1240706D5D40506D442F0080205E086
:100EB0009180C162F0BC704722F008028260998282
:100EC000012098711AE090F84A60D6B9104E766CFD
:100ED000B6F5966F15DC240713D49C8AB4F5FA6F27
:100EE00002D2641C9C82E5E70A4B65F3C3021C78BE
:100EF00024F001041C70598019828260F0BC08F053
:100F00000BB89982D6E7000070020020E2050020AD
:100F100038010020B00A0020012180F82E104FF483
:100F2000AF6101861F21418645F27151818670476C
:100F300070B506464089204B204C4FF400510025E7
:100F400080B362887AB1012A0CD1E188491C89B248
:100F5000E1803289914205D36580E580FF2801D088
:100F6000401E708170BD70882288904201D9012294
:100F700000E00022184602F0C4FB7088B1880144EA
:100F80002088401C80B220808142EBD82580A08838
:100F9000401C80B2A080F1888842E3D301206080A9
:100FA000A58070BDFFE70022184602F0AAFBA580CD
:100FB000E58025806580F4E700100140C805002029
:100FC000FEE7000010B5074C0021204600F06AF84B
:100FD0000121204600F066F82046BDE810400221BD
:100FE00000F060B80064004010B50D4C0B4920467D
:100FF00000F06AF809492046891C00F065F80949A3
:10100000204600F061F8084C206807F085FC0021BC
:1010100006A008F0DBFC206010BD00000200F0100C
:10102000006400407000F0304C0800206465765F7A
:1010300063616E310000000070B51848017861F3FB
:101040000704417861F30F24817861F31744C17874
:1010500061F31F640179407961F3070560F30F259F
:1010600002F0CEF80E4E304602F072F8A1B23046D1
:1010700002F0AAF8210CB01C02F0A6F8A9B2301DAB
:1010800002F0A2F805482838C07800F00301B01D2E
:1010900002F09AF8BDE8704002F08EB8A707002071
:1010A00000E4010841B101290AD0022903D1816875
:1010B00041F4000181607047816841F08001F9E7E7
:1010C000816841F40041F5E70A4A914202D10021CA
:1010D00081617047C1F313028B0101D5C260704773
:1010E0004B0101D502617047090101D5826070474B
:1010F000426070477000F03030B50823102404229D
:10110000B1F5007F1DD010DC202929D007DC012992
:1011100021D0042922D0082900D1C46030BD402943
:1011200020D0B1F5807FF9D10BE00025B1F5004F5B
:1011300006D008DCB1F5806F03D0B1F5006FEDD1BA
:101140008561426030BDB1F5803F0DD0B1F5003F03
:10115000F8D1446030BD0549816030BDC36030BD09
:10116000036130BD046130BD436030BD0101010049
:101170003EB5684600F026FA00208DF808000121EF
:101180008DF809108DF80A008DF80B108DF8060007
:101190001D498DF807008DF8020001F11000897CCF
:1011A0008DF80310C1788DF8041001798DF80510C1
:1011B000C088164CADF800006946204600F045F99D
:1011C00001220221204600F038F901221146204672
:1011D00000F033F90E492046FFF776FF0C49204610
:1011E000891CFFF771FF0B492046FFF76DFF084987
:1011F0002046491EFFF768FF01224FF404412046B4
:1012000000F01BF900203EBD5C0800200064004097
:101210000200F0107000F030094910B588424FF01C
:10122000010101D14C0601E04FF08064204604F03A
:10123000D3FC2046BDE81040002104F0CDBC0000E6
:10124000006400402DE9FF470026012119488DF870
:101250000B608DF80C10DFF86090ADF808608DF829
:101260000D10354634464FF0040809F1800AC7686E
:101270001AE000BF8DF80A4059F82610761C480B7A
:10128000ADF8000008EBC101ADF802105AF82510C6
:101290006D1C4A0BADF8042008EBC100ADF8060048
:1012A000684600F00BF8641CBC42E3DB04B000208D
:1012B000BDE8F08748080020B0180020F0B5827A19
:1012C000012191402E4A136843F0010313602C4B17
:1012D0001C331C688C431C60294D067B294C0C3543
:1012E000A6B92E688E432E604688C78846EA074610
:1012F000877A04EBC707C7F840660688878846EAFE
:101300000746877A04EBC707C7F84466067B012EB9
:1013100012D12E680E432E60867A056804EBC6064D
:101320004FEA3545C6F84056867A456804EBC60450
:101330004FEA3545C4F84456114CC57A241D002D9A
:10134000256806D00D4325600D4C0589143415B170
:1013500004E08D43F7E725688D4325600589012D5D
:1013600002D125680D432560407B012802D1186811
:1013700008431860106820F001001060F0BD000004
:1013800000660040006000400246002053690B42A6
:101390004AD0B1F5807F3BD013DC08292ED007DC82
:1013A000012926D0022927D004293DD1D0682BE07D
:1013B000102925D0202926D0402935D110691021A7
:1013C00030E0B1F5004F2BD00BDCB1F5007F22D01F
:1013D000B1F5806F22D0B1F5006F25D190697021F1
:1013E00020E0B1F5803F11D0B1F5003F1CD150682D
:1013F000E5E790680D4915E0D06802E0D068DEE7C7
:10140000106903210EE0106908210BE05068FBE72A
:101410009069012106E09069022103E0906900E0F3
:101420005068042100F0F6BF704700000101010080
:101430008069C0F3021000017047002A426901D0A0
:101440000A4300E08A434261704710B503680022F6
:1014500023F002030360036843F0010303604FF6C7
:10146000FF7300E0521C4468E40701D19A42F9D1AD
:101470004268D2073ED08A79012A02683CD022F025
:1014800080020260CA79012A026838D022F0400244
:1014900002600A7A012A026834D022F02002026037
:1014A0004A7A012A026830D022F0100202608A7A59
:1014B000012A02682CD022F008020260CA7A012AAE
:1014C000026828D022F0040202608A78CC78920761
:1014D00042EA04620C7942EA04424C79098842EA01
:1014E0000452491E0A43C261016821F001010160F2
:1014F000002114E0002010BD42F08002C1E742F05C
:101500004002C5E742F02002C9E742F01002CDE7F1
:1015100042F00802D1E742F00402D5E7491C4268D4
:10152000D20701D09942F9D14068C007E2D1012029
:1015300010BD000010B500EB0113D3F8B04114F05A
:1015400004041472D3F8B04134D0E408C2F8044063
:10155000D3F8B04104F002045472D3F8B44104F05B
:101560000F049472D3F8B441240AD474D3F8B84168
:10157000D472D3F8B841240A1473D3F8B841240CB8
:101580005473D3F8B841240E9473D3F8BC41D47388
:10159000D3F8BC41240A1474D3F8BC41240C54740D
:1015A000D3F8BC311B0E937439B1016941F02001AD
:1015B000016110BD640D1460CAE7C16841F02001EB
:1015C000C16010BD00218171C171017241728172CF
:1015D000C1728170C1700321017102214171012129
:1015E0000180704730B50246002093685B0108D443
:1015F0009068000101D5012003E09068C00037D554
:10160000022002EB0012D2F8803103F00103C2F88D
:1016100080310B7A73B3D2F880414D681C434B7A0A
:1016200043EAC5031C43C2F880418B7A03F00F03E1
:101630008B72D2F8843123F00F03C2F88431D2F8D0
:1016400084318C7A2343C2F88431CB7ACC6843EA64
:101650000423C2F88831CB7B096943EA0121C2F82F
:101660008C11D2F8801141F00101C2F8801130BD17
:10167000042030BDD2F880314C7A23430C8843EAF1
:101680004453C2F88031D0E72DE9F04FFE481A21CB
:101690008BB0406CDFF8F8B3B0FBF1F084B20D20F2
:1016A000B4FBF0F8F9485D46B0F91A00C0F30F102A
:1016B0000490BBF9100001F0C3F842F21071084425
:1016C000FEF7CAFEF34AF44BFEF7AFFDFEF709FF43
:1016D00080B20990B5F91E0001F0B2F80890B5F992
:1016E000200001F0ADF80790B5F9220001F0A8F84C
:1016F000EA4B0690D88B4FF4FA71484340F6FF71DD
:10170000B0FBF1F0DFF898C386B2E64DBCF81000EC
:10171000E5490190E8880A78070967F30002C70ADB
:1017200067F34102C70867F38202870867F3C302C1
:10173000070B67F30412470867F3451260F386123C
:10174000470B67F3C7120A704A78470A67F300022B
:10175000470967F34102870967F38202070A67F3C3
:10176000C302C70967F304122F7ABF0867F3451253
:10177000800B60F386124A7093F8070110B142F0B3
:10178000800001E022F080004870C6489A46827AC4
:10179000887862F341001A89D50885EA1225ED435D
:1017A00065F382009CF8005065F30410550965F359
:1017B0004510D20A62F386101A88D213521C62F3C3
:1017C000C71088709AF84A202AB1012A07D0022A45
:1017D0000AD0032A0DD0CA7822F003020CE0CA789E
:1017E00022F00302521C07E0CA7822F00302921C86
:1017F00002E0CA7842F00302AB4BCA702833A3F16F
:1018000018059A7802F00302012AAA7811D022F072
:101810001002AA70CA7897070ED020F008008870CE
:101820005879994600F00300012808D0022809D011
:101830000BE042F01002ECE740F00800EFE742F066
:10184000040001E022F00400C870974F2246791D81
:10185000F87820F09000F870381D05F04FF8934CA0
:10186000B4F9020005F0FDFEB871B4F9040005F00A
:10187000F8FEF87107F10804611C2046049A05F08F
:101880003DF8E11CA01C099A05F038F8884864214D
:10189000B0F904004843800B03F088F960713246C8
:1018A000E11DA01D05F02AF8BBF91000FFF76AFA48
:1018B000C8214843800B03F079F9287099F800009B
:1018C000012402274946B4EB901F03D1A87840F0C9
:1018D000010005E0B7EB901F03D1A87820F00100CC
:1018E000A8704B7803F00300012802D0022804D02E
:1018F00007E0A87840F0020002E0A87820F002009B
:10190000A870DAF80800AA784FEAD01C6CF38202BB
:10191000AA7091F802C05646CCF3810CBCF1010FBD
:1019200003D0BCF1020F03D005E042F0200201E039
:1019300022F02002AA70CB46A246B4EB931F03D13B
:10194000D1B241F0800104E0B7EB931F02D102F065
:101950007F01A9705749DFF84C91534C4A7FE978D1
:10196000183462F34101C20A62F3820196F82A2117
:1019700062F30001327962F3C301E97099F80A3029
:1019800029794A4663F3820133785B115B1C63F368
:10199000C301430963F30411297100166979401CDE
:1019A00060F3C301697199F80010E87961F30300ED
:1019B000D1884246C90B61F3861099F80810C9080E
:1019C00061F3C710E871611C204604F097FFE11C29
:1019D000A01C019A04F092FFB6F9E800FFF7D2F9D3
:1019E000C8214843800B03F0E1F82071307AC10927
:1019F000A07961F3C710B6F8C8100A0A62F30600AE
:101A0000A071E171273C611C2046089A04F076FF22
:101A1000E11CA01C079A04F071FF611D201D069AAD
:101A200004F06CFF84F806809BF800005C4620F010
:101A30000C00001D20F03000103020F0C0014031BB
:101A40008BF800109BF8010020F00300401C20F0F0
:101A50000C00001D20F0C00340338BF80130A0784B
:101A6000DFF844B020F00300401C20F00C00001D03
:101A7000A0708646E078ABF11F0B20F0E002403208
:101A8000E2709BF8000017E038010020D00400202D
:101A9000380500209A9999999999B93FA402002094
:101AA000B00A0020000C00207F070020F80D002065
:101AB000E2050020200E002000287DD0F07B0028C9
:101AC0007AD18BF800000BF1170090F800C00CF0F1
:101AD000030CBCF1010F06D090F800C00CF0030C11
:101AE000BCF1020F04D190F800C06CF30101217029
:101AF0000178C1F38101012904D00178C1F381018A
:101B0000022906D101784FEA910C21786CF3830108
:101B100021700178C1F30111012904D00178C1F3CA
:101B20000111022906D101784FEA111C21786CF3CA
:101B30000511217090F800C05146BAEB9C1F04D0EB
:101B400090F800C0B7EB9C1F09D190F800C04FEA95
:101B50001C1894F800C068F3871C84F800C090F843
:101B600001C00CF0030CBCF1010F06D090F801C0CD
:101B70000CF0030CBCF1020F04D190F801C06CF31F
:101B8000010363704378C3F38103012B04D04378CE
:101B9000C3F38103022B06D143784FEA930C637899
:101BA0006CF3830363704378C3F30113012B06D0F6
:101BB0004378C3F3011300E029E1022B06D14378F7
:101BC0004FEA131C63786CF3051363704378B1EB31
:101BD000931F03D04378B7EB931F06D143784FEAA6
:101BE000131C63786CF387136370837803F003032B
:101BF000012B04D0837803F00303022B05D190F866
:101C000002C073466CF30103A3708378C3F38103AE
:101C1000012B04D08378C3F38103022B06D1837890
:101C20004FEA930CA3786CF38303A3708378C3F318
:101C30000113012B04D08378C3F30113022B06D1C7
:101C400083784FEA131CA3786CF30413A370837892
:101C5000B1EB931F03D08378B7EB931F06D1837842
:101C6000C3F3011CA3786CF34713A370C378DB069E
:101C700008D0C37803F01F031F2B03D2C37863F38C
:101C80000402E270C278520905D0C2785309E278A2
:101C900063F34712E270027902F00302012A04D0D2
:101CA000027902F00302022A04D10279237962F355
:101CB000010323710279C2F38102012A04D002795F
:101CC000C2F38102022A05D102799308227963F3D3
:101CD000830222710279C2F30112012A04D002792F
:101CE000C2F30112022A05D102791309227963F3A2
:101CF000051222710279B1EB921F03D00279B7EB82
:101D0000921F05D102791309227963F38712227198
:101D1000427902F00302012A04D0427902F0030260
:101D2000022A04D14379627963F301026271427934
:101D3000C2F38102012A04D04279C2F38102022A4D
:101D400005D142799308627963F383026271427923
:101D5000C2F30112012A04D04279C2F30112022A0D
:101D600005D142791309627963F3051262714279F0
:101D7000B1EB921F03D04279B7EB921F05D14279A4
:101D80001309627963F387126271827902F00302A8
:101D9000012A04D0827902F00302022A04D1827956
:101DA000A37962F30103A3718279C2F38102012A4C
:101DB00004D08279C2F38102022A05D18279930884
:101DC000A27963F38302A2718279C2F30112012A1C
:101DD00004D08279C2F30112022A05D18279130953
:101DE000A27963F30512A2718279BAEB921F03D034
:101DF0008179B7EB911F05D181790A09A17962F345
:101E00008711A171C179E07961F30300E071434F5B
:101E1000387800F00F00042801D1FFF70DF9207881
:101E2000C0F38100012839D1F879010636D500F0D8
:101E30007F00142832D8A87840F00400A870384AEF
:101E4000A978107F8B074FF47F412BD5802821D3B1
:101E5000344B00F01F00126853F82000024219D1E1
:101E6000B06840F08070B0602C4830388078C0078F
:101E70001CD0B068C00119D52B48406C322815D849
:101E8000BBF8020088465C46404527D101F056FC6D
:101E900060800DE0B06820F08070E4E7A87820F062
:101EA0000400CBE7B06820F08070B060ABF802109F
:101EB000A878800702D40020A9F80A003879C00762
:101EC00001D0A9F80AA099F80A00C1071348A0F1A7
:101ED0004900017812D041F0010111E001F016FC37
:101EE00040F6B8318842E3D3B068C101E0D50005BF
:101EF000DED4A9F80AA0A4F80280D9E721F00101F4
:101F00000170B168C901017802D541F0020101E018
:101F100021F0020101700BB0BDE8F08FAF07002087
:101F2000E80500202CB400083801002070B51548E1
:101F3000006810F0E05F23D0134CD4E90010814218
:101F40001ED004EB001104F5A1608A6842600A7B90
:101F5000827204230372002545720B300E31FEF7A6
:101F600012F972B66068401C6060402800D365605A
:101F700062B60649BDE8704002480838FFF732BB38
:101F800070BD000008640040A8140020B0190020B3
:101F9000FCB505464FF6FF7600200C46ADF8006014
:101FA00048F205078DF8040020E000BF15F8010B8A
:101FB0008DF8040001A9084602F084FBBDF800007A
:101FC0009DF8041080EA0120ADF800005FF00000E9
:101FD000BDF800100A0402D587EA410101E006EAD3
:101FE0004101401CADF800100828F1DB641EDDD271
:101FF0006946084602F050FBBDF80000FCBD000039
:102000000246002004E000BF12F8013B1844C0B2B1
:10201000491EF9D27047000070B5144A85B0108887
:1020200000241349019400940394204604941388D7
:1020300007E0CD8B009E354400950D8B019E354405
:10204000019515889D42F4D0401CC0B28028EED383
:102050000098411107484180848001984111064849
:1020600081830183818205B070BD00004807002094
:10207000A4020020E2050020D004002030B4104C5F
:10208000002003464FF47F42A4F1340121F81030C0
:1020900024F81020401C1A28F8DB0A4B002000BF4F
:1020A00033F8104021F81040401C1A28F8DB06488D
:1020B00006490280012081F8300030BC03F054B999
:1020C0006C100020080800203C080020CC0E0020E6
:1020D0002DE9F84303F094F9C64DC54B00204FF4A9
:1020E0007F4105F1340400BF35F8106033F810204B
:1020F000964203D025F8102024F81010401C1A280E
:10210000F2DBBD4890F83000012808D05FF00000F5
:1021100024F81010401C1A28FADBBDE8F88302F0FE
:10212000F5FD208801F0F2FA2988B44E88420AD3DE
:1021300001F004FB2080B24800906B460822B149B0
:10214000306808F0A9FE608801F0E0FA69888842EA
:102150000CD301F0F3FA6080A948AA49401C009012
:102160006B4608220831306808F096FEA08801F01E
:10217000CDFAA98888420CD301F0E0FAA080A048EB
:10218000A049801C00906B4608221031306808F08E
:1021900083FEE08801F0BAFAE98888420CD301F0A6
:1021A000CDFAE08096489749C01C00906B46082203
:1021B0001831306808F070FE208901F0A7FA2989EB
:1021C00088420CD301F0BAFA20818D488D49001D58
:1021D00000906B4608222031306808F05DFE60896F
:1021E00001F094FA698988420CD301F0A7FA608162
:1021F00083488449401D00906B460822283130688E
:1022000008F04AFEA08901F081FAA846A9890527AD
:102210007D4D884216D36878052813D201F08EFAD6
:10222000A0816878401CC0B26870052800D96F7022
:1022300073487449303000906B4608223031306862
:1022400008F02AFEE08901F061FAB8F80E10884221
:1022500016D3A878052813D201F070FAE081A87887
:10226000401CC0B2A870052800D9AF706448654909
:10227000313000906B4608223831306808F00CFE8F
:10228000208A01F043FAB8F81010884216D3E87893
:10229000052813D201F052FA2082E878401CC0B21F
:1022A000E870052800D9EF70554856493230009043
:1022B0006B4608224031306808F0EEFD608A01F07C
:1022C00025FAB8F81210884216D32879052813D2B7
:1022D00001F034FA60822879401CC0B228710528C8
:1022E00000D92F7146484749333000906B46082289
:1022F0004831306808F0D0FD208D01F007FAB8F8B9
:102300002810474688420BD301F018FA20853F4831
:102310003C4900906B460822A031306808F0BCFDB3
:10232000608D01F0F3F9798D88420CD301F006FA43
:10233000608536483349401C00906B460822A8311E
:10234000306808F0A9FDA08D01F0E0F9B98D884250
:102350000CD301F0F3F9A08529482A4950300090A8
:102360006B460822B031306808F096FDE08D01F030
:10237000CDF9F98D88420CD301F0E0F9E0852048D1
:102380002049603000906B460822B831306808F070
:1023900083FD208E01F0BAF9398E88420CD301F00A
:1023A000CDF9208616481749613000906B46082207
:1023B000C031306808F070FD608E01F0A7F9798EA9
:1023C00088420CD301F0BAF960860D480D4962309D
:1023D00000906B460822C831306808F05DFD0C485B
:1023E000FFF726F800283FF498AE287095E6000025
:1023F0000808002038100020CC0E00204C080020D7
:102400000002FF18000F0020400800200006FF18FF
:1024100000640040024600200A4200D001207047BC
:1024200030B50E4902880A800C4A4388083A138066
:102430000B1F808818802024151F2C800020401C32
:1024400080B23C28FBD341F69910088044F648003E
:10245000108046F6480018802C8030BD202C0140AA
:10246000114944F648000880091D46F648000880D6
:10247000091D41F6991008800B48001F018841F0A2
:102480002001018009480021A0F86810A0F866101A
:10249000A0F86410A0F86210A0F86010A0F85E1018
:1024A0000348418181827047182C0140A40200201A
:1024B0004C0000202DE9F04F4B4B4C480021DA7ABC
:1024C0000678802A26F001057AD31C68484B02F072
:1024D0001F0253F82220474B14421A6802D042F0E0
:1024E000200201E022F020029946DFF80CB11A60C8
:1024F000434B404F9BF80040DFF800A1B3F9043094
:1025000097F84AC0022C5CD1D9F80870C7F3C00410
:10251000C7F30028444554D0364C343C94F802802C
:10252000B8F1000F06D0B8F1010F0DD0B8F1020FCD
:102530004CD120E0110549D5910647D40121A17065
:1025400026F00401017041E015053FD495063DD504
:1025500075073BD4458895BB4380002B09DD46F0C9
:10256000050101700221A1702649B1F844100182D1
:102570002CE0A1702AE0C6880EB9002B14DC067B83
:10258000664511D1204EB6895FEA46780CD45FEAE1
:10259000867809D45FEA427806D55FEA826803D577
:1025A000F60701D1FE0111D505704180AAF800108F
:1025B00041810182A17089F80F108BF8001005E0AD
:1025C0000EE005704180AAF800104181C38080F8B8
:1025D0000CC0500960F3CB22C9F80020BDE8F08F91
:1025E000057041804181F9E7E8050020B00A00202C
:1025F0002CB40008A40200203F0700200C0100209A
:10260000E205002038010020000C00202DE9F047F1
:1026100096B000240C940D940E940F9472B68048DA
:10262000816941F400718161816941F48061816156
:102630004FF4004003F0AEFA7A4D00212846FEF731
:1026400045F900212846FEF737F9774E002130463C
:10265000FEF732F9754F0021384600F06FF901207E
:102660004FF47041401C8842FCD32846FEF750FAD4
:10267000B1463046FEF74CFA384600F06BF94FF49D
:102680006020CDE912048DF8454001204FF0040888
:102690008DF8440010948DF8508010A92846FEF75C
:1026A000C9FA01231A4605212846FEF714FB012327
:1026B000022206212846FEF70EFB012303220721F2
:1026C0002846FEF708FB012304220F212846FEF7C7
:1026D00002FB384600F03EF9684600F0DEF951484A
:1026E000534E4C300090CDF80C80CDE90164802031
:1026F000CDE904404000069080000790202008901B
:102700004FF44050CDE909046946384600F0A8F975
:1027100001212846FEF7DAF80121384600F00EF9CB
:1027200001212846FEF7C8F847F230501594159954
:10273000491C15918142FAD301212846FEF70AFB74
:10274000ADF82C40A04640F2DC5A4FF4007420E073
:102750005046CDF854801599491C15918142FAD301
:1027600030880D9908440D9070880E9908440E9099
:10277000B0880F9908440F90F0880C9908440C9089
:1027800001212846FEF7E6FABDF82C00401CADF802
:102790002C00BDF82C00A042DAD30D98C1112448BA
:1027A0000A3001830E99C91141830F99C9118183A0
:1027B0000C99C91181801F49C988490407D41E4951
:1027C000028B21F85C2F428B4A80808B888000210D
:1027D0002846FEF77BF80021384600F0AFF80021CC
:1027E0002846FEF769F800214C464846FEF764F893
:1027F0000220C102401C8842FCD32846FEF788F91B
:102800002046FEF785F9384600F0A4F8FEF768F890
:102810000A493C20087062B616B0BDE8F087000097
:10282000001002400024014000280140080002403E
:102830002E050020000C0020580E00203C07002030
:1028400010B5FEF79FFA4FF42F614843800B10BD7F
:1028500070B5204B40F6C81441F2B7055B6C48F6E2
:10286000E6065C4305EBA4341B4D73434EF6F616A7
:1028700006EBA333C5E90443D460401A53611060EA
:102880009168884202DA4942884200DC116010688F
:102890004343107E0341906A19189162506A814245
:1028A00000DD9062916A106A814201DB084600E017
:1028B0009062A86111684C43117C0C4108412118B9
:1028C000B2F91C00884204DBB2F91A00884200DC2D
:1028D00008B270BD380100201401002010B54FF47B
:1028E0000054204600F0ACF8002813D00A490878BC
:1028F00040F008000870204600F014F80021074856
:1029000000F01CF80648C17E012903D10021C176E0
:102910000121017710BD0000820600204400024022
:10292000040D0020C10002D5024908607047024929
:10293000486070470404024000000240002901681A
:1029400002D041F0010102E04FF6FE721140016039
:102950007047000001684FF6FE72114001600021CF
:10296000016041608160C1603149314A083990425B
:1029700003D1486840F00F0006E02D4A143290421F
:1029800004D1486840F0F00048607047284A283277
:10299000904203D1486840F47060F5E7244A3C3225
:1029A000904203D1486840F47040EDE7204A50322D
:1029B000904203D1486840F47020E5E71C4A643235
:1029C000904203D1486840F47000DDE7184A78323D
:1029D000904203D1486840F07060D5E7154A111F56
:1029E000904203D1086840F00F0006E0114A14320B
:1029F000904204D1086840F0F000086070470D4A2A
:102A00002832904203D1086840F47060F5E7094A23
:102A10003C32904203D1086840F47040EDE7054A2B
:102A200050329042EAD1086840F47020E5E7000097
:102A30000800024008040240406880B2704700006D
:102A400001460020CA0001D5034A00E0034A12688B
:102A50000A4200D0012070470004024000000240FA
:102A600030B5036847F6F07293430C6A8A682243D4
:102A7000D1E904452C4322438C692243CC6922438B
:102A80004C6A22438C6A22431A430260CA6842603D
:102A90000A6882604968C16030BD00210160416000
:102AA0008160C160016141618161C1610162416216
:102AB0008162704710B5114C8CB000212046FFF7A1
:102AC0003DFF2046FFF746FF0D4800900D480021CE
:102AD000CDE901016420CDE903018020CDE90501A4
:102AE0000791089109910A9169462046FFF7B8FFBE
:102AF00001212046FFF722FF0CB010BD5800024014
:102B000004380140F0080020F0B540F6AA222A4916
:102B1000C284838B0C88E31A9BB20F2B0DD30988D8
:102B20008183037E00213BB1244BB3F90A40244B3F
:102B3000062C03DA818429E08184F0BD214C2478BD
:102B4000022C02D0002CF5D0F0BD1F4C40F68B2794
:102B5000656C1B4CA5F22D16BE42B4F9004017D28D
:102B6000418B491C89B241836429EDD3642141839F
:102B7000B0F92410914201DA01EB22128284641C24
:102B800020B24FF4007118808842DDDB1980F0BD5F
:102B900041F29416B542FADBB0F92450002D02DD63
:102BA000A5EB221200E0002282844183641E20B241
:102BB00018800028EADDF0BD480700204C00002006
:102BC000540400203F0700203801002010B50446BF
:102BD000B0F9020043F6991148438113E06840F2CE
:102BE0006662504301EBA030E060B4F9001043F698
:102BF000991251438A13216940F26663594302EBEB
:102C0000A131216105F032FC6061A18840F6AB2260
:102C100008444010A0F515415539E062914205D9AC
:102C2000A0F5F851FF39521C91421DD249F254517E
:102C3000884202DDA0F5204002E0A0F5F850FF3800
:102C4000206300EB400040F34F002085B4F92410CE
:102C50004A42904201DA104602E0884200DD08460E
:102C6000E083228461848AE0A0F5FE42FF3A41F2CB
:102C700055518A4214D8A2F6AA20206300EB4000E6
:102C800040F34F002085B4F924205142E18388426B
:102C900001DA084602E0904200DD1046404250E072
:102CA000A0F5D442AA3A8A4215D2A2F6AA202063FD
:102CB00000EB400040F34F012185B4F9240042426B
:102CC000E2832084914201DA104602E0814200DC76
:102CD0000846608453E0A0F5AA42543A41F25653A4
:102CE0009A4215D2A2F6AB20206300EB400040F3DD
:102CF0004F002085B4F924104A42904201DA104670
:102D000002E0884200DD08464042E083218419E069
:102D1000A0F5804241F254539A4215D2A2F6AA205D
:102D2000206300EB400040F34F002085B4F92410ED
:102D3000E1834A42904201DA104602E0884200DD17
:102D40000846208462841AE0A0F52852AB3A8A42F1
:102D500015D2A2F6AA20206300EB400040F34F01F9
:102D60002185B4F92400E08342422284914201DAB1
:102D7000104602E0814200DC08464042A9E7B4F96F
:102D80001E0041420948B0F9000041438913E18027
:102D9000B4F920104942414389132181B4F922102A
:102DA000494241438813608110BD00005404002053
:102DB00000210176704770471548164A4FF480414C
:102DC0000078042821D002F13C03D08A9B88C01AE5
:102DD00000B22F2801DD001108E0002801DD0020ED
:102DE00007E00D4B984201DA184602E0402800DD6A
:102DF00040209389184400B2884203DC40F26661A7
:102E0000884200DA0846908170479181704700003F
:102E10003F070020D0040020C0FEFFFF38B54B481C
:102E20004B4902880B889A1A92B20F2A71D30988EB
:102E3000484C01804FF0FF01E2884FF47A7355044B
:102E40004FF4967002D51622009103E0950403D545
:102E500015220091014670E0D50402D5142200919C
:102E6000F8E7150502D513220091F3E7550502D5C1
:102E700012220091EEE7950502D511220091E9E7B3
:102E8000D50502D510220091E4E7150602D50F22E0
:102E90000091DFE7550602D50E220091DAE795068C
:102EA00002D50D220091D5E7D50602D50C2200915E
:102EB000D0E7150702D50B220091CBE7550702D5C5
:102EC0000A220091C6E7950702D509220091C1E7C1
:102ED000D20702D008220091BCE72289550702D50B
:102EE00007220091B6E7950702D506220091B1E7C7
:102EF000D20702D005220091ACE7A27AD20702D015
:102F000004220091A6E7A289D40603D503220091EA
:102F1000A0E719E0140702D5022200919AE75407AE
:102F200003D4940701D4D20702D00122009191E783
:102F30000020034602460146009003F0FBFBBDE87B
:102F400038400248FDF7F4BF38BD0000F40B002004
:102F500048070020000C0020F0B5594859498288E4
:102F60000B889A1A92B29C2A64D3098881805649A8
:102F70000A880146002A0B7843F0020156D1164612
:102F8000524A1C0715680246127822F0020274D5D4
:102F90004F4C0746E4887F785FEA845C02D547F0AF
:102FA000010701E027F001074770A704477802D521
:102FB00047F0020701E027F002074770670401D4D9
:102FC000E70703D0477847F008074770640603D542
:102FD000447844F0040404E01C0603D4447824F04C
:102FE00004044470EC0450D4354C9A07247824F03F
:102FF000100423D4324D42782F7A2D78012A45F0DF
:10300000100514D0022A16D02D4C042AA47804F1FD
:10301000010C0CF0FF0C13D0072A25D0032A23D073
:10302000052A21D0062A1FD021F0100142E0B9075D
:1030300002E00570F0BD39070029FADB0470F0BD2D
:10304000FA0601D41A060AD50170022C04D280F8BF
:1030500002C0BCF1020FF2D341F080012AE021F05E
:10306000100101708670F0BD877A7F06F7D5032CBA
:1030700004D8017080F802C0F0BD0FE05107D8D528
:103080001906D6D443F0800114E002704178CB07D2
:1030900001D18907F0D522F010010BE0E9040BD42F
:1030A0009907E9D4818AC82902D2491C8182E3E7C1
:1030B00043F00A010170DFE702708682DCE700005E
:1030C00010070020480700204A070020A402002023
:1030D000000C002070B51148114C4FF00005C0885D
:1030E000810503D4410601D4C00515D54FF4806194
:1030F0000C4800F0FBFA68B9A08840F6B831884265
:1031000001D2401CA08080B2B0F57A7F01D30120AB
:10311000607070BDA58070BD6570FBE7000C00207D
:1031200060070020000C0140084946F6680008804E
:10313000091D0880091D41F6DD5008800348001F65
:10314000018841F02001018070470000182C0140E7
:1031500070B50D4E0546304600F05EF8042811D1DA
:103160000A4C206940F0020020616561206940F04E
:1031700040002061304600F04FF8216941F6FD72B1
:103180001140216170BD0000FFFF0F0000200240D0
:1031900008490420CA68D20701D001207047CA68D4
:1031A000520701D502207047C968C906FBD5032024
:1031B00070470000002002400248016941F0800190
:1031C0000161704700200240F0B506464FF6FF77D8
:1031D0000D46384600F020F804280DD1074C206930
:1031E00040F0010020613580384600F015F8216973
:1031F00041F6FE7211402161F0BD00000020024046
:103200000348024941600349416070472301674513
:1032100000200240AB89EFCD00B50346FFF7B8FFB1
:1032200003E000BFFFF7B4FF5B1E012803D0002BB3
:1032300000D1052000BD002BF4D1FAE710B5C288FB
:1032400000210AB1032206E002890AB1022202E04B
:10325000428912B10122027000E0017004784FF43B
:10326000804344F6206244B1012C06D0022C07D0E2
:10327000032C01D14180818010BD4380828010BD2C
:1032800041F23331418040F6B731F4E7401A106023
:103290009168884202DA4942884200DC1160516933
:1032A0001068137E41431941936A0B449362516A3B
:1032B0008B4200DD9162936A116A8B4200DA91625F
:1032C000D168936A4143107C01410341B2F91C006B
:1032D0001944884204DBB2F91A00884200DC08B2C3
:1032E00070470000054920B1086940F0800008617E
:1032F0007047034848600348486070470020024018
:1033000023016745AB89EFCD06494FF47A70CA684F
:10331000D20705D0401E0004000CF8D1FF207047F2
:1033200000207047002002400E4A0320A2F14C0109
:1033300082F83E000020C8800B490886C862C88316
:103340000884488490620948016DB1F5206F01DB63
:10335000A3219162807A002802D0906A4042906254
:10336000704700004C000020380500203801002084
:10337000F0B53D4988894A89801A80B20F286AD3FE
:1033800088894881CA8939480B3A272A26D28A78FF
:1033900022BB8268384B42F480728260344A374CD8
:1033A000374D12785607334A0AD4364E368816807F
:1033B000354A12881A80354A12882280344A09E038
:1033C000344E36881680344A12881A80334A12885E
:1033D0002280334A12882A8001228A70314A0021D1
:1033E000314B82F84D1019469A7F304D0968802A7A
:1033F00032D302F01F0255F8222011422CD08268ED
:1034000022F48012184E8260123614461215B778D4
:10341000521C62F38617264AB77093F816C01778C5
:10342000BCF1800F27F0020608D30CF01F0C55F8F2
:103430002CC011EA0C0F01D147F0020616701A7E5B
:10344000802A0DD302F01F0255F82220114207D125
:1034500044F400218160F0BD826842F48012D1E71B
:1034600024F40021F6E700003C070020A40200201D
:1034700038010020C8040020CA040020CC04002029
:10348000CE040020B8040020BA040020BC040020B0
:10349000BE040020C0040020C2040020C404002098
:1034A000C6040020580E0020E80500202CB40008B7
:1034B000D004002070B5214881890289891A89B217
:1034C0000F2932D381891E4D1E4C0181697A2268F1
:1034D0001D4E42F00400802908D301F01F012B6823
:1034E00056F821100B4201D122F004002060FFF7B2
:1034F000F1FDA87B802819D300F01F00296856F839
:103500002000014212D1206820F002002060E87AF9
:1035100080280FD300F01F00296856F820000142D0
:1035200008D1206820F00800206070BD206840F0BD
:103530000200EBE7206840F00800F5E73C070020B8
:10354000E8050020A40200202CB4000830B5044691
:1035500000204FF40043024640EA030101FB01F55D
:10356000A54200D80846521C5B0812B2102AF3DBB1
:1035700030BD0000F0B51D4C1B4A4FF0010C94F813
:103580003B5094F80AE0144692F83C3094F83840E6
:103590002B43651CEEB2154D95F83D700025BEF12C
:1035A000FF0F0AD0BEF1000F06D18B4213D1557028
:1035B0000C2C01D282F83860F0BD834202D182F82F
:1035C00001C0F5E78B42F7D15570B80709E000BF9D
:1035D00082F83850F0BD8342FCD1F84382F801C034
:1035E00080070028F4D0F0BD5804002038010020E6
:1035F000F0B5CA78002502F00F03D20601D58A780B
:1036000013430A784FF00F0E12F0FF0F4FF0010234
:103610001CD004680F8802FA05F63740B74211D172
:103620004FEA850C0EFA0CF724EA070703FA0CF4AC
:103630003C43CF78282F02D0482F02D002E04661C9
:1036400000E006616D1C082DE4D304600C88FF2C9B
:103650001ED944685FF0000606F1080702FA07F574
:103660000F882F40AF420FD14FEA860C0EFA0CF7AD
:10367000BC4303FA0CF73C43CF78282F00D14561B7
:10368000CF78482F00D10561761C082EE4D3446022
:10369000F0BD0000F0B5144C002801DAE36900E049
:1036A0006368420D120185B2C0F301579540C0F323
:1036B0000346032F05D0C2020AD50322B24093432A
:1036C00007E023F07062636823F07063636002E0D8
:1036D000AB4343F0706201B12A43002801DAE26192
:1036E000F0BD6260F0BD0000000001400246002015
:1036F00092680A4200D00120704741617047016121
:1037000070470AB101617047416170474FF6FF622F
:10371000B0F57F4F04D0911C884203D10020704740
:103720001046704704490988814201D3081A01E014
:10373000101A084480B270478808002001480088A9
:1037400070470000880800200F4A104B92F838108C
:103750005B5C834201D1012004E00D4B5B5C834242
:1037600003D1002082F83A0070470A4B5B5C834229
:1037700001D18120F6E7084B595C814201D18020BC
:10378000F0E70320EEE7000038010020E4B800086D
:10379000F6B80008EAB80008FCB800080A4810B5F6
:1037A00001784FF000024C0708494FF0FF03896889
:1037B0004FEA017105D5002901DA827210BD8372CA
:1037C00010BD0029FBDBF8E738010020A40200202F
:1037D000F0B5194E194C0022E31CA6F1060CB75C9B
:1037E000A518ED78FF5C0D430F43BD421FD01CF8B8
:1037F0000270FF5C0F43BD4219D015460023A61886
:10380000F6780E43C6545B1C1CF80220DBB2062B74
:10381000F5D3C17881700179C17000214218491C2B
:1038200015711CF80550C9B20629F7D3F0BD521C1A
:10383000D2B2032AD3D3F0BDBEAF00085804002093
:1038400010B502460021064B06205C1864789442AD
:1038500000D10846491CC9B20629F6D310BD0000A4
:10386000380100200548D0E900218A4202D14FF0FA
:10387000FF30704700EB011080687047A0100020F7
:1038800070B5164C05464FF0FF36D4E90010814262
:1038900021D004EB001080686860606804EB0010C1
:1038A000007B00F00F02AA7204202872606804EB0B
:1038B000001105F10B000E31FCF765FC72B6606873
:1038C000401C6060402801D30020606062B6A87A86
:1038D00008B1002070BD304670BD0000A01000206F
:1038E00030B526484FF000028078C107244840D008
:1038F00024498988E9BB2449234B40F6B834496CF4
:10390000B3F87630A14231DD90F84A1071B31F4907
:10391000C9790C062AD501F07F015A2926D290F8E0
:103920002B11491CC9B280F82B11C8291ED380F86D
:103930002B21D0F83041014604F1640591F82C1197
:10394000AB4203DD052908D2491C01E041B1491E03
:1039500080F82C11C9B2052902D3012180F82A115F
:10396000191B074C343CE162C0F83031B3F5FA6FF3
:1039700003D280F82A2180F82C2130BD8F07002047
:10398000A4020020E205002038010020AF0700203B
:103990004FF42032C260002181620E22028241F285
:1039A00062024261082202834FF4604242838183B3
:1039B0004FF07842C0E9082140F6C41101807047F9
:1039C000B0F90010B0F90220891A41604269037E03
:1039D0004A431A41836A13448362426A934200DD78
:1039E0008262836A026A934200DA8262C268836AF0
:1039F0004A43017C0A410B41D118B0F91C208A428C
:103A000001DA10467047B0F91A008842FADC08B2B1
:103A10007047000010B514481449B0F894200B8882
:103A20009A1A92B2B2F5437F1DD90988A0F8941072
:103A3000B0F8921020F8601F002242860C480D4C0E
:103A4000C2888280C180C38983812489891AA4B2F3
:103A5000C4818160E11A0161074A818AC182928A28
:103A60008282511A816110BD380100204807002070
:103A7000200E0020380500204C00002009480A498B
:103A8000B0F8B2200B889A1A92B241F684639A4237
:103A900006D3098820F8B21F418881800021418027
:103AA0007047000038010020480700200D480178C9
:103AB000C90702D00C49098801E04FF6FA71416646
:103AC000094901201039088007482438018841F04D
:103AD0000101018004481838018821F01801018093
:103AE0007047000038010020240400400A49D1F842
:103AF000982012B1521EC1F8982031F8922F521C12
:103B000021F81A294A6A521C4A628A8F521C8A87F3
:103B100001F8400C70470000380100201CB52D480A
:103B200090F83B3090F83C20934252D000248DF81E
:103B3000044053408DF800309DF800300122012BE5
:103B400008D09DF80030022B09D09DF80030042BDE
:103B50000AD00DE01F498DF80420443108E01D49CA
:103B60008DF80420463103E01A498DF804204831CD
:103B70009DF80420012A2CD190F83D309DF800409A
:103B8000154AA34217D090F83E309DF800402342DA
:103B900008D0B0F84C30A0F84A300B881488E31AEB
:103BA000A0F84C3090F838302BB1B0F84030148881
:103BB000E31AA0F8423012880A80A0F8402010F8DA
:103BC0003E1F9DF80020114300F801199DF80010D8
:103BD00001701CBD580400204807002070B5344D0A
:103BE00040212846FFF782FD840080212846FFF708
:103BF0007DFD44EA4004A9152846FFF777FD0443FC
:103C0000E1B22C4C94F878508D4250D04D4084F85D
:103C10007810012D03D0022D01D0042D47D194F846
:103C20007C00A84384F87C0094F87B20AA420FD043
:103C300084F87B5094F87A2001238B401A4207D1F4
:103C40001A4384F87A2094F87910491C84F8791082
:103C500094F87910042928D330B1012811D0022812
:103C60000FD004280DD012E01348C18821F0400184
:103C7000C1802078002184F83B1020F06000207083
:103C800005E0217841F02001217084F83B000B49C8
:103C900094F83B0091F82720904204D081F8270047
:103CA00007492020087000F00DF884F8545070BDCA
:103CB0000010014038010020000C0020580E0020A8
:103CC0003C07002070B50D4D40212846FFF70EFD42
:103CD000840080212846FFF709FD44EA4004A91525
:103CE0002846FFF703FD04430548072100F8784FF5
:103CF0000171002141708170C17070BD00100140E0
:103D00003801002070B5344890F83A10CA43920741
:103D100061D001F0030280F8392090F83D305B0655
:103D20001B0E80F83D30012A01D0812A02D15B1C94
:103D300080F83D300278D2074DD0DBB203F00102AB
:103D4000C3F34004A24246D1B0F856400025641C9B
:103D5000A0F85640204CA0F8585090F83E60A47A45
:103D6000B24202D080F83E200DE0A607B6EB837F7A
:103D700002D080F83F5006E090F83F30642B02D22A
:103D80005B1C80F83F3090F84030642B0CD25B1CF9
:103D9000DBB280F84030022B06D204F001039342DC
:103DA00002D1022280F84020012901D0002912D13D
:103DB00090F83820416E00EB820291610163D0E9F6
:103DC00006121144D0E908231A441144826A1144AE
:103DD000C26A1144416370BD38010020FEE7000053
:103DE0002DE9F04F00BF00209E4E9F4AA6F51271AC
:103DF000A6F5BE79A6F1440B06F1440E804601F506
:103E0000E074A1F1780301F5457A1D5C15F0C00757
:103E100006D0402F51D0C02F77D0802F76D004E12C
:103E200015F01F0504D0154440F080072F7201E003
:103E300082F80880012826D0022824D0032822D026
:103E4000042820D008281ED010281CD0874D55F8F3
:103E500020C0DCF8005054F820703D40CCF80050F1
:103E6000824D55F820C0DCF8005056F820703D43D4
:103E7000CCF800501D5CAD0659F820502F6813D5C2
:103E80003AF810C03EE051F820502F6854F820C096
:103E900007EA0C072F6051F820502F6856F820C011
:103EA00047EA0C072F60E5E7DFF8B8C10CF1F00C2A
:103EB0005CF820C007EA0C077EE015F01F0504D06F
:103EC000154440F080072F7201E082F80880012835
:103ED0001DD002281BD0032819D0042817D0082889
:103EE00015D0102813D0614D55F820502F6854F884
:103EF00020C007EA0C072F605C4D55F820502F6852
:103F00005BF820C047EA0C0756E00BE056E051F89A
:103F100020502F6854F820C007EA0C072F6051F892
:103F20002050ECE715F01F0505D0154440F0800740
:103F300085F8217001E082F82180012825D002282F
:103F400023D0032821D004281FD008281DD01028F2
:103F50001BD0464D55F820C0DCF8005054F82070B6
:103F60003D40CCF80050414D55F820C0DCF80050E1
:103F70005EF820703D43CCF800501D5CAD0615D5B1
:103F80003A4D3AF81070CC3514E051F820502F68B3
:103F900054F820C007EA0C072F6051F820502F6812
:103FA0005EF820C047EA0C072F60E6E72D4D3AF88F
:103FB0001070E03D55F820502F6036E015F01F05D9
:103FC00005D0154440F0800785F8217001E082F8A3
:103FD0002180012830D002282ED003282CD004289C
:103FE0002AD0082828D0102826D0204D55F820C0E7
:103FF000DCF8005054F820703D40CCF800501B4DC8
:1040000055F820C0DCF80050164F883757F820705C
:104010003D43CCF800501D5CAD06B1D4114F3AF8C9
:104020001050E03F57F820703D60401CC0B211288E
:10403000FFF4EBAEBDE8F08F51F820502F6854F834
:1040400020C007EA0C072F6051F820502F68DFF8D6
:1040500014C00CF1880C5CF820C047EA0C072F60F4
:10406000D9E70000B8B60008E8050020B4B400089D
:104070004FF40771C1824FF45861018340F6145127
:1040800081837047F0B5C48AB0F900608681B0F9C9
:104090000250C581B0F904300227002101220382B9
:1040A000AB4204DBB54202DDC78042810CE0B34283
:1040B00004DBAE4202DDC78041811CE09D4205DB8E
:1040C000B34203DDC2804781018115E0B54204DBC4
:1040D0009E4202DDC280418105E0AE4205DB9D4289
:1040E00003DDC1804281078106E09E4204DBAB42D2
:1040F00002DDC18047810281C388458900EB430707
:1041000000EB4505BB89AE899B1B0FFA83FEA0F827
:1041100012E00689AB8900EB460CBCF80CC0A3EB9F
:104120000C038382B0F91830B7F90CC0A3EB0C0C68
:10413000B4EB4C0F04DA80F82010A3F1A10113E0D6
:10414000A64503DD80F82010B9890BE026B1012EC9
:1041500004D0022E10D004E0062100E0052180F8F2
:104160002010A989091B6D31418309B2B1F5586F3F
:1041700004DB5B1E438304E00421F0E7002900DC3C
:104180004283418B8183F0BD0B49002288760A620D
:10419000CA614A62094A32F9103002EB40028B626E
:1041A000B2F90220CA62064A32F810000882A1F869
:1041B0006000A1F862007047F00100200EB900080D
:1041C00002B900082DE9F05FFE48FF4982880B889C
:1041D0009A1A92B20F2A45D309888180FB498246F8
:1041E000FB4D0888FB4F4FF00108002678B3401EB6
:1041F0000880EE73F849EE622868B1F902104307AF
:1042000042F6AA2218D4FB8843F40053FB80F24BF9
:104210001B789B0709D5AB6823F08003AB60A5F83A
:10422000806085F8826085F88360C30404D485F8D3
:10423000F480C5F8F06003E085F8F460430707D424
:10424000914205DB85F8F880A5F8F66004E010E0FF
:1042500085F8F860430703D4914201DBC00703D01F
:1042600085F81561BDE8F09F85F81581A5F8166100
:10427000F8E7B5F81C0143F69821884202D2401CA9
:10428000A5F81C0102F06CFADFF85093DFF834B3A4
:1042900099F85000ABF1180B10B1FEF70BF905E0DF
:1042A0009BF8001021F001018BF80010FFF718FBBC
:1042B00000F01EFACA4841F26802416C4FF40060F7
:1042C000914201DBC74A04E0B1F57A6F02DAC54AD0
:1042D000121D1060C148DFF8F8920A2490F85100CE
:1042E000DFF804C3C007A9F1340938D09CF80E00E8
:1042F000802802D32878800705D5BC480078C206FC
:1043000001D4800627D5EA7B89F80720B24A4846BF
:10431000137823F002031370ABF802609BF80030AF
:1043200023F001038BF80030BA7952060FD482894A
:10433000B2F5FA7F03D2521CA9F80C200FE040F628
:104340003C70814201DD002467E0042465E0002424
:10435000A9F80C6061E089F80360A9F80C60A8680E
:10436000020501D5082458E09C4A92F83FE05FEA34
:10437000CE7247D0EA7B89F807209CF80930802B61
:1043800045D39B4B9B781B0641D52B785B0732D4DA
:10439000FB889B0404D500BF20F02000A86031E01A
:1043A000ABF802609BF8004040F0200024F00104CC
:1043B0008BF80040A8609CF8170080280BD300F011
:1043C0007F044FF00040DCF80030E040034202D1AF
:1043D00085F8048000E02E712879C00702D15FEAD9
:1043E0008E7005D50324032A17D089F80A8014E0BB
:1043F0000024EE6211E020F02000A860F88820F48C
:104400000050F88095F82A01012805D005E02A68B7
:1044100042F004022A60BFE7092408B2754903F09C
:1044200057FB6B49744DCA6A50438013A1F8E800EA
:104430000A2C6FD16E488078800602D5FCF718FDF3
:1044400009E063488168CA0502D521F0080101E04E
:1044500041F0080181605E484FF40054620090F81A
:104460004A8042F6CC4142F26663B8F1010F1FD098
:10447000B8F1020F31D02978DFF880C1B8F1030F0D
:10448000C1F381013CD043F6FE7801293FD00229D7
:104490003DD0A0F8182100BFA0F8482047F23C31D9
:1044A000ACF800104D4991F87010012933D03FE06D
:1044B00095F800C0CCF3810CBCF1010F07D0BCF122
:1044C000020F07D0A0F81811A0F84810EAE7A0F8EA
:1044D0001831F9E7A0F81841F6E795F800C0CCF3D9
:1044E000810CBCF1010F08D0BCF1020F05D0A0F87F
:1044F000182100BFA0F84820D4E7A0F81811F9E768
:10450000A0F81821A0F8482046F65471C8E7A0F892
:104510001881C1E77BE02978C1F3810101290ED020
:1045200002290FD041F6E121A0F81811A0F8483077
:104530009BF80030DB0708D0BBF8103007E0A0F88C
:104540001831F3E7A0F81841F0E723498B88AAF85F
:10455000123019B2B0F948305943C1F38F3349468C
:10456000A9F81830934200D90A83254A1278D20656
:1045700005D50B8B41F23332934200D20A83826815
:10458000C2F3C003C2F30024A34205D10C8B41F651
:1045900099139C4200D90B831A4B9B78DB0707D0F9
:1045A000D20105D4114A127802F00F02032A00D07A
:1045B0000E83B9F81810C162002927DD12480224C1
:1045C000067024E0C80A0020480700204A0700209F
:1045D000A4020020000C0020E2050020580E00205C
:1045E00038010020100C0140E8050020AF07002032
:1045F0008F07002008AF0008D00400203001002001
:10460000100700207F0700205C07002000249AF894
:104610001A0098B9022C30D084B11B480278930656
:1046200008D5BB795B0605D5184B1B78DB0963F30E
:1046300086120270F88820F40A60F8801248406CF4
:104640004E2815DBFB88180612D5B9F81620521C27
:1046500092B2A9F81620B2F5FA6F04D3A9F8166041
:1046600023F08000F8800A48027822F002020270EB
:1046700008488AF81A40C473F4E5288F0028CCD182
:1046800043F698202887C8E738010020100700204B
:10469000E2050020A402002070B500230C8863F31B
:1046A0000F02012505FA03F6344206D0C3F10F06C6
:1046B00005FA06F1114361F30F025B1C102BF1DBCD
:1046C000028070BD70B500230C7863F307020125EA
:1046D00005FA03F6344206D0C3F1070605FA06F1DF
:1046E000114361F307025B1C082BF1DB027070BD04
:1046F000F0B5204890F866101F480129836823F41C
:10470000006234D11D49CE88740630D41C4D1F057B
:104710004FF00004B5F9025020D41A4A526C642AB2
:1047200011DC40F6386295420DDAB2040BD40278FF
:10473000520710D4B0F8D82040F6B835AA4203D2B8
:10474000521CA0F8D820F0BD43F400628260D00172
:10475000F9D44C81F0BDA0F8D840F0BD41F2CD03B2
:104760009D42FADD897AC907F7D18260F3E782605A
:10477000F0BD0000580E0020A4020020000C002014
:10478000E205002038010020F0B5364D364F0446D2
:1047900095F83B0097F83B1023780843EE1C6278AD
:1047A000834205D1E0781146FEF7E4FE207908E067
:1047B00094F802C084450CD1E1781046FEF7DAFE89
:1047C000E07905F82F0F2878805D6870287BE877FE
:1047D000F0BD82421DD161461846FEF7CBFE95F82A
:1047E0004E1095F83B00814207D1B97A09B1A17901
:1047F00000E0617985F82F101EE06978012901D069
:10480000A17922E0617927E0297841F0040129703B
:1048100012E0E1788142DBD119466046FEF7AAFE3C
:1048200095F84E1095F83B0081420AD1B97A09B14A
:10483000617ADFE7217ADDE715F82F1F895D69705E
:10484000C5E76978012906D0617A85F82F10B97A11
:104850000029F1D1D8E7217A85F82F10B97A0029FB
:10486000EAD0D1E758040020380100200B48017835
:1048700021F0020100F8381B002100F818194177D7
:10488000817733218185418508214184012100F808
:104890001F1C034880F8391070470000580400209E
:1048A000380100200D4900B50B4851F8012F40F8A0
:1048B000032F89888180084801210930FEF788FF8D
:1048C000054802211330FEF783FF034804211D3001
:1048D0005DF804EBFEF77CBF58040020380100208F
:1048E000094944F648000880091D46F6480008803A
:1048F000091D41F2111008800348001F018841F092
:104900002001018070470000182C01402DE9F0477C
:10491000664C674B0025A0780126654A10330528B0
:104920007ED2DFE800F00313113E1100108820F062
:10493000010010801D805F480580001F0580001F5A
:104940000580FFF7CDFFA670BDE8F087594941F615
:10495000CC401C390880574945F658002439088056
:10496000091D46F658000880524920202839088041
:104970000020401CC0B27328FBD3FFF7B1FF4C49A5
:1049800084F85C502C3147F6906008804848143019
:1049900006801D80108840F0010010800220A07069
:1049A000D2E700215FF0010004EB410204EB400379
:1049B000B2F85020B3F850309A4200D20146401C61
:1049C000C0B20628F0D33C48405C84F83900FFF7B9
:1049D0004DFF1D2000F0B0FD00F076F8374E38484E
:1049E0004FF4807996F83B10012904D002291BD09E
:1049F000042930D047E040218046FEF777FE87004B
:104A000080214046FEF772FE47EA4007494640468D
:104A1000FEF76CFE074347F0010084F83B0000E01E
:104A20003DE0224809302CE040218046FEF75EFE42
:104A3000870080214046FEF759FE47EA4007494675
:104A40004046FEF753FE074347F0020084F83B0060
:104A50001648133015E040218046FEF747FE8700D8
:104A600080214046FEF742FE47EA4007494640465D
:104A7000FEF73CFE074347F0040084F83B000B4878
:104A80001D3003F021FB94F82F0086F838001D201C
:104A900000F068FD0420A0700A48057054E71088F3
:104AA00020F0010010801D80A5704DE75804002003
:104AB000000800403C2C0140C4AF00083801002031
:104AC000001001403F0700202DE9F041344C14F85C
:104AD0002F0F344DE07240212846FEF707FE860076
:104AE00080212846FEF702FE46EA4006AF15394609
:104AF0002846FEF7FBFD0643207BF1B22F3C8142A6
:104B000015D084F83C0040212846FEF7EFFD8600D2
:104B100080212846FEF7EAFD46EA40063946284647
:104B2000FEF7E4FD064384F83B60FEF7F7FF1E4DF9
:104B300095F83B00012827D0022828D0042829D046
:104B4000174894F83B102730085C04F8300F14F82D
:104B50000109FEF775FE04F82F09A87A00B10120BB
:104B6000607001F0A5FE94F84E0094F83B10884266
:104B700006D094F83800062802D2401C84F8380089
:104B800084F84E10BDE8F0810548093004E004487F
:104B9000133001E002481D30BDE8F041FFF7F4BDDD
:104BA000580400200010014038010020FF2801D9DE
:104BB000FF207047C0B270472DE9F0414A4991F893
:104BC0007200AA2874D191F87300552870D1474C0F
:104BD00000200A5C2254401CC0B27428F9D3444E11
:104BE0002069C6F80100A08AA6F80500D4F81600CE
:104BF000F060D4F81A003061D4F81E0012347061ED
:104C000003F008FA3B49608A888103F01DFA207D91
:104C1000123CC007307802D040F0040001E020F0E0
:104C20000400354930704FF480400861334D14F86A
:104C3000280F334985F82000608B6880A08BA880FE
:104C4000E08BE880208C2881608C688194F82400B7
:104C500081F8D60014F8010C86F83B000027C6F84E
:104C60009C70FFF71FFE2748A18E0183E18E4183D0
:104C7000218F818394F84210283C012908D0022911
:104C800001D0032909D0297821F00C01083107E06F
:104C9000297821F00C01091D02E0297841F00C016E
:104CA000297094F8642018491AB101224A8101E060
:104CB0000EE04F8194F8701001290BD094F86D101C
:104CC00059B101290CD04FF4805100BFA0F87610E3
:104CD000BDE8F08144F21C71F8E74FF40051F5E7AC
:104CE00041F25551F2E7000000FC0008580E002088
:104CF000380100204C000020F80D0020D0040020D6
:104D0000A402002038050020000C002010B5FCF79C
:104D1000BBFCFE48FE4AFF49807AC00703D0887872
:104D200020F0010005E09078800703D0887840F0FB
:104D300001008870F8480B7803704B7843708B78CB
:104D40008370CB78C3700B7903714B7943718B7986
:104D50008371C979C171EF49083109780172ED4950
:104D6000083149784172EB49083189788172E94903
:104D70000831C978C172E749083109790173E549F9
:104D8000083149794173E349083189798173E149EF
:104D90000831C979C173DF49103109780174DD49DF
:104DA000103149784174DB49103189788174D949CF
:104DB0001031C978C174D749103109790175D549C5
:104DC000103149794175D349103189798175D149BB
:104DD0001031C979C175CF4918310B7803764B78FA
:104DE00043768B788376CB78C3760B7903774B79D0
:104DF00043778B798377C979C177C6490F390978A9
:104E000080F82010C3490F39497880F82110C14932
:104E10000F39897880F82210BE490F39C97880F897
:104E20002310BC490F39097980F82410B9490F398A
:104E3000497980F82510B7490F39897980F826100B
:104E4000B44920310B7880F828304B7880F829302D
:104E50008B7880F82A30CB7880F82B300B7980F86B
:104E60002C304B7980F82D308B7980F82E30C97931
:104E700080F82F1000F1D001097880F8301000F18F
:104E8000D001497880F8311000F1D001897880F89C
:104E9000321000F1D001C97880F8331000F1D00150
:104EA000097980F8341000F1D001497980F8351083
:104EB00000F1D001897980F8361000F1D001C9796C
:104EC00080F8371000F1D001097A80F8381000F12D
:104ED000D001497A80F8391000F1D001897A80F840
:104EE0003A1000F1D001C97A80F83B1000F1D001EE
:104EF000097B80F83C1000F1D001497B80F83D101F
:104F000000F1D001897B80F83E1000F1D001C97B0F
:104F100080F83F1000F1D001097C80F8401000F1CA
:104F2000D001497C80F8411000F1D001897C80F8E3
:104F3000421000F1D001C97C80F8431000F1D0018B
:104F4000097D80F8441000F1D001497D80F84510BA
:104F500000F1D001897D80F8461000F1D001C97DB3
:104F600080F8471000F1D001097E80F8481000F168
:104F7000D001497E80F8491000F1D001897E80F887
:104F80004A1000F1D001C97E80F84B1000F1D00129
:104F9000097F80F84C1000F1D001497F80F84D1056
:104FA00000F1D001897F80F84E1000F1D001C97F57
:104FB00080F84F1000F1F0010B7880F850304B78FA
:104FC00080F851308B7880F85230CB7880F85330AD
:104FD0000B7980F854304B7980F855308B7980F814
:104FE0005630CB7980F857300B7A80F858304B7AAE
:104FF00080F859308B7A80F85A30CB7A80F85B3061
:105000000B7B80F85C304B7B80F85D308B7B80F8CD
:105010005E30CB7B80F85F300B7C80F860304B7C5F
:1050200080F861308B7C80F86230CB7C80F8633014
:105030000B7D80F864304B7D80F865308B7D80F887
:105040006630CB7D80F867300B7E80F868304B7E11
:1050500080F869308B7E80F86A30CB7E80F86B30C8
:105060000B7F80F86C304B7F80F86D308B7F80F841
:105070006E30C97F80F86F10264950310B7880F868
:1050800070304B7880F871308B7880F87230CB7844
:1050900080F873300B7980F874304B7980F8753074
:1050A0008B7980F87630C97980F87710117880F89C
:1050B0008010517880F88110917801F0030180F818
:1050C0008210117980F88310517980F884109179D9
:1050D00080F88510D17980F88610117A80F88710D1
:1050E0000C4938310A7802F0030280F888204A78A7
:1050F00080F889208A7880F88A20CA7880F88B2006
:105100000A7980F88C204A7908E00000000C002021
:10511000101000207F070020000F002080F88D2055
:105120008A7980F88E20C97980F88F106B490A78C7
:1051300080F890204A7880F891208A7880F8922030
:10514000CA7880F893200A7980F894204A7980F808
:1051500095208A7980F89620C97980F897105F4960
:1051600008310A7880F898204A7880F899208A785F
:1051700080F89A20CA7880F89B200A7980F89C20D1
:105180004A7980F89D208A7980F89E20C97980F834
:105190009F10524918310A7880F8A0204A7880F888
:1051A000A1208A7880F8A220CA7880F8A3200A7902
:1051B00080F8A4204A79C2F3400363F35F0280F8C9
:1051C000A5208A7980F8A620C97980F8A7104349DC
:1051D00020310A7802F0010280F8A8204A7880F88D
:1051E000A9208A7880F8AA20CA7880F8AB200A79AA
:1051F00080F8AC204A7980F8AD208A7980F8AE201A
:10520000C97980F8AF10354928310A7880F8B02084
:105210004A7880F8B1208A7802F0030280F8B22040
:10522000CA7880F8B3200A7980F8B4204A7980F8E7
:10523000B5208A7980F8B620C97980F8B710274957
:1052400030310A7880F8B8204A7880F8B9208A7816
:1052500080F8BA20CA7880F8BB200A7980F8BC2090
:105260004A7980F8BD208A7980F8BE20C97980F813
:10527000BF101A4938310A7880F8C0204A7880F87F
:10528000C1208A7880F8C220CA7880F8C3200A79C1
:1052900080F8C4204A7980F8C5208A7980F8C62031
:1052A000C97980F8C7100D4940310A7880F8C820C4
:1052B0004A7880F8C9208A7880F8CA20CA7880F8AD
:1052C000CB200A7980F8CC204A7980F8CD208A79E1
:1052D00080F8CE20C97980F8CF1010BDBF0700201C
:1052E0007CB50121082000F083FC4FF40050ADF89C
:1052F000040010248DF8074001208DF8060001A954
:105300001548FEF775F90121092000F071FC012113
:105310001248FEF7BFF90820ADF8000004208DF810
:1053200003000F4E03258DF8025069463046FEF704
:105330005FF908213046FEF7E0F9ADF800408DF83E
:1053400003408DF8025069463046FEF751F91021AE
:105350003046FEF7D2F97CBD001401400002300057
:10536000000C0140FEE7000038B50121082000F0E4
:105370003FFC4FF44060ADF8000048208DF803007A
:1053800003201B4D8DF8020069462846FEF730F9D0
:1053900029152846FEF7AAF9164CE914607020700A
:1053A0002846FEF7A3F9E070A070FEF7C7F9A080C9
:1053B000E080114890F84A10104849B101290BD0FB
:1053C00002290FD003290CD1C17841F0030107E075
:1053D000C17821F0030103E0C17821F00301491CE9
:1053E000C17038BDC17821F00301891CF8E70000C5
:1053F000000C014080080020A40200207F0700204C
:105400002DE9F041414D4FF480612846FEF76EF9D9
:105410000446E9142846FEF769F9DFF8F4800746E8
:10542000002598F800002E46844205D088F80040F8
:10543000FEF784F9A8F8040098F80100844209D026
:10544000B8F80400FEF762F91E2803D388F801407B
:10545000A4B3002598F802004446874203D0A77001
:10546000FEF76CF9E080E078874207D0E088FEF72D
:105470004DF91E2802D3E7701FB300266078254936
:10548000002808791FD020F002000871E278EAB104
:1054900020F0010008710DB1002E2DD155EA060053
:1054A0002AD01D4BDA7802F00300032800D903202C
:1054B000002475B103280CD2401C10E0FFE7012541
:1054C000C8E70126DAE740F00200DEE740F001001D
:1054D000E0E726B118B1012810D0401EC0B260F339
:1054E00001020E49DA7070B1012803D0022801D000
:1054F000032801D181F84A00BDE8F0818978C90606
:10550000EDD50020EBE781F84A40F5E7000C0140BB
:10551000800800208F0700207F070020A4020020C1
:10552000704700F01F02012191404009800000F106
:10553000E020C0F88011704700F01F020121914067
:105540004009800000F1E020C0F88011704700F0B1
:105550001F02012191404009800000F1E020C0F8C5
:105560000011704700F01F020121914040098000A6
:1055700000F1E020C0F800117047000070B50F2363
:10558000C47801780122F4B1144C2468457804F4FD
:10559000E064C4F5E064240AC4F10406E3408478BE
:1055A000B5401C402C4301F1E021230181F8003477
:1055B000007800F01F018A404009800000F1E020DF
:1055C000C0F8002170BD01F01F0082404809800032
:1055D00000F1E020C0F8802170BD00000CED00E07B
:1055E0000249084302490860704700000000FA05BC
:1055F0000CED00E02DE9F05F00261D20FFF791FF84
:105600006C4CDFF8B4B1A4F1B800A77E90F8381064
:10561000DFF8A8E1DFF8A8A100258F427ED0E77669
:10562000A176626A036B5A434FEA12499BF808203D
:10563000120702D51EF8012000E00A4694F812C0B5
:10564000BCF1010F09D004EB4206B6F902C0C4F860
:1056500028C0B6F90460E6620CE043F6FF7CC4E9BA
:105660000A5C90F83DC05FEACC7C01D012B102E048
:10567000052A00D1012600EB47074FF0804CBF8977
:105680003F04B7FBF3F3E361476BBCFBF7F727621B
:1056900094F813C0BCF1000F06D0BCF1010F05D087
:1056A0003B4403EBD3735B10636201E03B466762EC
:1056B000DFF810C14FF6FF7707EA8307ACF80870F0
:1056C0009AF8007090F80A8090F83DC0082F08F012
:1056D00003070CF0030C05D067450BD1B8F1000FA0
:1056E00005D008E0674505D0B8F1000F03D05B4254
:1056F000636200E06562C6B1636A002B03D006DD19
:10570000228D05E00AE0304B33F8122000E0A28D34
:10571000A4F86020227822F0200222709AF800205B
:10572000042A07D0082A05D012E0B4F8603003EB51
:105730000902EDE780F8405065629BF80800000719
:1057400001D51EF80110204830F81100A4F86000BF
:105750001E49606A09883E314843B4F8601001EB85
:10576000204006B21D20FFF7F2FE606A002807D035
:1057700021784FEA81600ADD002804DAA08D09E073
:10578000B4F8600006E0E06AB04208DB0CE00028F4
:1057900002DA208D208208E0A06AB04204DD208277
:1057A00041F02000207000E0268225756575258671
:1057B000BDE8F09FF0010020A4020020F0B800082E
:1057C0003F070020940B002002B900082404004089
:1057D00043184FF48042934210DD904202DD1046A0
:1057E00000210BE0914202DD0020114606E080031B
:1057F000B0FBF3F000B2C0F5804109B241EA0040CD
:105800007047F0B541F2F1130022C3600E248262AA
:1058100004824BF2660508264561068343F6FF774E
:105820004283878340F2492E4FEA873CC0F808E064
:10583000C0E9082CCB608A620C824D610E834A83DA
:105840008F83B4208860C1E9082CF0BD00218162FB
:105850000949C1600E210182084941610821018383
:105860004FF44041418343F6FF7181830907016290
:105870000349416270470000B6A001001C0C010002
:1058800000C0FF0F064941F68160088005480168A5
:10589000054A01F4E06111430160BFF34F8FFEE759
:1058A000442C01400CED00E00400FA05F8B501219C
:1058B0000D2000F09DF94FF4E060ADF800001824D1
:1058C0001D4E8DF8034003258DF802506946304681
:1058D000FDF78EFEB1153046FDF70FFF711530460E
:1058E000FDF70BFF31153046FDF707FF4FF4604021
:1058F000ADF800008DF80340104C8DF80250694659
:105900002046FDF775FE61142046FDF7F8FE4FF4C2
:1059100080412046FDF7F3FE4FF400412046FDF79D
:10592000EEFEA014ADF8000048208DF80300694693
:105930002046FDF75DFEF8BD00080140000C014067
:105940002DE9F0410121CE028CB0304600F050F933
:10595000DFF87081404601F03BFC08A801F064FECE
:105960004FF45860ADF824000024ADF8204020200A
:10597000ADF822000125ADF826408DF8285008A981
:10598000404601F003FE0021404601F056FE4FF66E
:10599000FF71404601F05BFE01220021404601F00C
:1059A000E7FD0121404601F0CFFB04A801F0E7FB31
:1059B000ADF81060A802ADF81200ADF814408120D7
:1059C000ADF816002803ADF81800ADF81A40ADF890
:1059D0001C4004A9404601F0C1FBADF80840082076
:1059E000ADF80A006027ADF80C408001ADF80070FA
:1059F000ADF80440ADF80E00ADF80240ADF8064039
:105A00006946404601F0A4FC6946404601F0E6FCC8
:105A10006946404601F02CFDADF8045040F61450A4
:105A2000ADF80070ADF80600ADF80840ADF80C40D8
:105A3000ADF80250ADF80A40ADF80E406946404658
:105A400001F05AFD0121404601F0A2FB0821404629
:105A500001F0BEFC3146404601F000FD0821404601
:105A600001F044FD3146404601F078FD702140468A
:105A700001F081FD18208DF82C008DF82D408DF857
:105A80002E408DF82F500BA8FFF778FD0D480C30F5
:105A9000018841F0800101800A481430018841F0FA
:105AA00001010180001F04800121404601F07AFBC2
:105AB0008DF828500121404601F07EFB0CB0BDE876
:105AC000F0810000002C0140704740F2134141601A
:105AD000082181608621C1604FF480410161494203
:105AE000416100210162C16270470162704700009C
:105AF00010B501884288891A09B20183B1F5005FA7
:105B000002DBA1F5804104E011F5005F02DC01F544
:105B100080410183B0F9182041685143C161836815
:105B2000846A5343C2681B12624303EB2222036A56
:105B30001A44114402628A13426241698A4203DBB9
:105B400001698A4200DC11468A1AC0E90A21028EE4
:105B50004FF40373594302EBA13202860B4A1278C9
:105B6000082A04D10A4A936F03EBA1319167B0F977
:105B70003010B1F5804F02DDA1F5804103E000292E
:105B800002DA01F58041018610BD00003F070020C8
:105B9000140C0020034A516821F440410143516034
:105BA0007047000000100240044A0029516901D0EA
:105BB000014300E081435161704700000010024042
:105BC000044A0029D16901D0014300E08143D16139
:105BD0007047000000100240044A0029116901D0FA
:105BE000014300E081431161704700000010024052
:105BF000044A0029916901D0014300E08143916189
:105C00007047000000100240044A0029D16801D00A
:105C1000014300E08143D160704700000010024062
:105C20002DE9F041274CA61540212046FDF75EFDE9
:105C3000850080212046FDF759FD45EA40053146A3
:105C40002046FDF753FD0543EDB240212046FDF708
:105C50004DFD870080212046FDF748FD47EA4007BB
:105C600031462046FDF742FD0743F8B2A842DBD19A
:105C700040212046FDF73AFD870080212046FDF7B0
:105C800035FD47EA400731462046FDF72FFD074323
:105C9000F8B2A842C8D140212046FDF727FD870071
:105CA00080212046FDF722FD47EA40073146204685
:105CB000FDF71CFD0743F8B2A842B5D12846BDE860
:105CC000F08100000010014010B50268416802FB3D
:105CD00002F301FB0133B3F1805F11D91B0E103BBE
:105CE0000A4C9BB212B234F8133009B25A435943EA
:105CF00042F38F3241F38F31C0E90221012102E0EA
:105D0000C0E902210021017410BD0000DCAE0008D2
:105D10002DE9F05FFE48FF4902880B889A1A92B27B
:105D20000F2A7DD309880180FB490A468889D288D9
:105D3000430703D4830701D4C30702D042F400729F
:105D400001E022F40072CA808A46010702D451465B
:105D5000C00606D5BAF8061041F00101AAF80610EF
:105D600004E0C88820F00100AAF80600EA48FDF720
:105D700065FAEA48B0F93A10B1F5804F02DA491CE9
:105D8000418703E0E5494FF480404887DFF890936E
:105D900041F6CC40E349D9F85020824203DD8868BF
:105DA00020F010008860E04BE04E0024188820B1FD
:105DB000401E1880CC73347029E0BAF80600450400
:105DC0001DD4BAF80C30DD0619D41D0717D405060A
:105DD00015D4850613D4050511D4450603D5D44D35
:105DE0002D782D060BD5450709D4C50507D4050721
:105DF00005D4850403D4C00601D4D80707D0CD4804
:105E0000CC73CD4B3470C4831C8080F828408B4603
:105E1000B1F84210DFF82483C94869B1491E00E097
:105E2000ECE0ABF8421098F8005025F0020588F835
:105E300000508BF80F400BE098F8003043F002035D
:105E400088F800303178012903D10178062900D182
:105E500034703178DFF8ECE2BB4D01270A2973D2A8
:105E6000DFE801F0FDCC05CCFCFBCC72FAF902F0C6
:105E7000E7F9DFF8B0A2AA48AAF1340ABAF81C1070
:105E8000491C8AB2AAF81C20416C40F628208142A5
:105E900002DAAAF81C4013E0A04840F6CC43C068E0
:105EA00098420DDBB8F9040043F69913984207DBDA
:105EB000B2F5FA7F04D32A7812B9AAF81C402F70E1
:105EC000A24A108868B19AF804305B1CDBB28AF8E9
:105ED0000430022B05D39E488AF8044003885B1CDB
:105EE00003809BF80F00D846092814D002287DD0E3
:105EF000A8F83441B8F84400DFF858B2A146C8B158
:105F000041F288344846AAF81C90A14221DA297847
:105F100001291AD01DE07E484430FDF739FDFDF718
:105F200003FA7F48416CCAF8301041F27C51CAF83C
:105F300020108FE2A88AA8F83400E86A6863A86A8B
:105F40002863A8F8447040E0C6E1814928700880C1
:105F5000108098F84A10022908D09BF80310B7EB7C
:105F6000511F10D098F82C1151B104E098F82C1161
:105F700009B96FF0A200C8F8DC0088F8EE7008E0FC
:105F80006FF40560F7E7C8F8DC0088F8EE00CAF89F
:105F900028009BF80300B8F93410B7EB501F05D068
:105FA000B8F8DC00102300B21A460AE001F21D50D6
:105FB00040F63A22904201D8102300E0202310221C
:105FC000002000F0C3FBA8F834009BF803006249EE
:105FD000B7EB501F52484FF49A73406C10D0B0F595
:105FE000FA7F0BDAB5F90A00984200E023E005DCFD
:105FF00086F8009088F8EE90A1F81A90BDE8F09F1E
:1060000040F2DC52904203DAB5F90A209A42EFDD01
:10601000B8F8442040F6C413521C92B2A8F84420A9
:106020009A42E5D23D4AD268002AE7DC42F6E062B5
:106030009042DDDAE2E7B8F8340140F6B832904237
:1060400007D2334B183B1B78DB0702D1401CA8F862
:10605000340183B204E0D4E0B2E0F9E0F4E0FCE023
:1060600040F2DC50834202D842F6CC4003E0A8F86C
:10607000342143F26660E867CAF830108AF8097084
:10608000364EA8F8444088F8EE40707F5546F8B187
:10609000F07FD8B3B8F82C00B8F9341000B20A2356
:1060A000052200F053FBA8F83400F47786F81D4071
:1060B000B8F91A01B8F9181188426CDA697901F156
:1060C000010111F0FF0169716CD06C71401C64E03A
:1060D0004FF48040A8F8E800D8F82C10814200DA8C
:1060E00008461F4900B2688391F84D1051B998F8DD
:1060F0004A1039B1B8F80820C2F3C003C2F3002235
:10610000934231D1B8F9341036232BE03FE0000040
:10611000C80A002048070020000C00203805002095
:1061200038010020A40200204C0700203F07002077
:1061300010070020300A002006000020E2050020A1
:1061400040070020580200204C00002008000020DA
:106150000A000020A70700203C0B0020200E002092
:10616000580E0020052209E0012903D0022901D0A0
:10617000032906D0B8F93410DA23242200F0E6FA15
:1061800006E0B8F9341040F299135122F6E7A32043
:10619000A8F834008CE703DD801EA8F81A0101E09E
:1061A000A8F81A11B8F934004FF48041884202DD92
:1061B000A8F8341022E70028FCDAA8F834401DE7DC
:1061C000D84ADBF8E0105846914202D2491CC0F888
:1061D000E010C17B082903D1D0F8E01091420CD324
:1061E00034708168CA0502D521F0080101E041F050
:1061F00008018160CBF8E04000E7BDE8F05F02F005
:106200009DBF9BF80F005F46092803D0BC868BF822
:106210000F4061E1C44D686A401C6862022809DDD4
:10622000288E012301B2288C052200B200F08EFADC
:106230006C622863BD48298E0180B9F84410418002
:10624000FDF7BEFBB886D9E6BDE8F05F04F0E6BC1A
:106250009EF8000009287DD0D0E68BF811419BF80C
:106260002C3163B142F31101CBF8DC40B04A8B030F
:10627000E962891093628A03A962AE498A62AA49D7
:106280008C83D9F8442041F288318A4207DA297890
:10629000012904D1A8492C700C80A8490C80A84A77
:1062A000DFF8A0C21188491C8BB2A7491380C82B04
:1062B00004D391F80080B8F1010F19D0B3F57A7FBB
:1062C00004D391F80080B8F1020F11D0B3F5FA6F42
:1062D00002D30B78032B0BD09BF80F10891E0829D3
:1062E0007ED2DFE801F010B9FBF7047D85AB85E6CF
:1062F0000C701480BAF8062022F40062AAF8062076
:106300008CF80070E8E7D9F84410C846822904DA0E
:106310000178062901D00470F5E0FDF73FFA98F8FE
:106320000000400613D58948807804280FD0D8F89B
:106330004410404682290ADA817A98F83D0001F03B
:10634000030100F00300814201D001F029FEB146B3
:10635000307800E0C0E00628C9D088F83F40D8F87F
:106360005000734940F311008203E86280108A6292
:106370008103A8626F4846468162FCF7D5FF6A48F0
:106380005D464772BBF81801ABF81A01706CABF8A8
:106390008640B0F5437F10DD4FF48040A5F88400BF
:1063A000A86840F48060A86096F8381005299ED14E
:1063B00040F01000CBF8080016E04FF48041A5F83B
:1063C0008410A96821F48061A96040F28A21884282
:1063D00004DA3078400601D402F09EFDA86800E09F
:1063E00098E040F01000A860022089F8000005E65F
:1063F000D9F84410B1F5437F02DA017806298AD131
:106400005348017821F040010170FCF78DFF43F6FD
:10641000FE70ABF81A010BF1E005FDF7BFF94D482E
:1064200010F8341F21F00101017042492C608C6288
:106430003F498C62082131704464DFE53B48FDF739
:10644000A7FAFCF771FF3848D9F84410016341F20C
:106450007C51016209203BE09AF80600C006C6D4D0
:10646000D9F844004D46B0F57A7F35DDFDF796F951
:106470002878400611D53548807804280DD0686CFE
:1064800082280ADAA87A95F83D1000F0030001F09E
:106490000301884201D001F083FD85F83F40B5F843
:1064A0005000ABF8340001B24FF480405C468142AA
:1064B00000DDA086FCF738FFA06840F48060A06093
:1064C00095F83810052992D140F01000A060022004
:1064D000307093E514E001E034708FE5D9F8441092
:1064E000B1F5437F02DA0178062988D1BAF806109F
:1064F00021F02001AAF80610FDF750F90420E7E783
:106500000078062801D0377078E509208EF8000061
:106510000520DDE70D498C70047085F85E40ABF80E
:1065200034406BE5C0D40100700200200C0B002049
:10653000000A0020D00900200A00002008000020E6
:10654000100100200E01002012010020580400203C
:106550004E070020140C002030B585B00121042026
:10656000FFF746FB4FF40040ADF8100048208DF8CF
:10657000130004A91848FDF73BF801210846FFF76E
:106580001FFB40F68C20ADF8040003240020ADF87A
:106590000040ADF80200ADF806004FF080456946B6
:1065A000284600F0F3FF1C208DF80C008DF80D40FC
:1065B0008DF80E4001208DF80F0003A8FEF7DEFFD6
:1065C00001221146284600F0BBFE0121284600F0BA
:1065D000E9FD05B030BD0000000801407047000033
:1065E0002DE9F041304CE07800285AD1207800287D
:1065F00057D0401E10F0FF00207052D14FF496701B
:10660000208272B6294F45F2AA50A7F872000020E6
:10661000FCF768FE264D13202860FCF775FEA8BB2A
:106620003420E86002202861224E6E61286940F023
:1066300040002861FCF768FE40BB00211E4A084666
:106640005FEA255312F800C0BCF1FF0F00D0012112
:10665000401C80B29842F5D3C1B9C4E90676392608
:106660000127A06910F8011B10F8012BA061E06957
:1066700001EB022102886A612F6120F8021BE061B0
:10668000FCF742FE10B9761EB6B2EAD20120FCF742
:1066900029FE62B601F0D8FC0848816821F48041E7
:1066A0008160BDE8F08100003C070020580E00200A
:1066B0000020024000FC000800FC0008A4020020AA
:1066C0001948016841F010010160016821F00301DF
:1066D0000160016841F002010160144841684160B5
:1066E00041684160416841F480614160416821F442
:1066F0007C11416041680E4A11434160016841F0DC
:106700008071016001688901FCD5416821F00301B5
:106710004160416841F0020141604168C1F381017B
:106720000229FAD170470000002002400010024008
:106730000000280830B5044C039D6080A180E280F1
:106740002381658130BD0000F40B00200A448242A1
:1067500001DA10B27047C91A8142FBDD08B27047F6
:106760002DE9F04F4A48DFF82CA1DFF82CB1C17FAA
:10677000477A046849480022DFF82C91466C484863
:106780004FF0010E802985784648836834D301F0A4
:106790001F0C5AF82C100C420146096802D041F433
:1067A000805101E021F4805101605FEAC14C1ED4A8
:1067B0005FEA814C1BD599F80AC0C8465FEACC7CD9
:1067C0000BD05FEAC31C12D4A8F80A209BF8008003
:1067D00028F002088BF8008009E0322E07DC5FEA1F
:1067E000857C04D55FEA035C01D4A8F80AE04FEA8F
:1067F000113C6CF34D310160802F24D307F01F074B
:106800005AF827100C42016802D041F0040101E05F
:1068100021F0040101604C0711D44C050FD599F803
:106820000A70FF070BD0DF0109D4A9F80A209BF8F2
:10683000007027F002078BF80070C0F89C208C08CD
:1068400064F38A21016099F80A40E40719D1174CD2
:1068500094F86440012C14D1322E10DC04686607D1
:106860000DD51B050BD4E30409D5AB0707D5D0F82C
:106870009C304EF66024A34205D9A9F80AE0C0F87E
:106880009C20BDE8F08F5B1CC0F89C30F9E700004D
:10689000E80500202CB40008E205002038010020A3
:1068A0008F070020A4020020000C0020580E0020BA
:1068B00010B5FAF773FA0F48018821F00201018040
:1068C0000C49183109880C4A928E1144094A343215
:1068D000118008490C390A8842F001020A80011D22
:1068E0000A884FF6ED531A400A80018841F01201E0
:1068F000018010BD0C04004058040020130A0370EE
:106900000A70704705484FF6FF620188491C89B23A
:106910000180914201D30021018070478808002046
:106920000F4810B5016841F00101016041680D4A4E
:106930001140416001680C4A11400160016821F476
:1069400080210160416821F4FE0141604FF41F0184
:106950008160FFF7B5FE05494FF00060086010BD8B
:10696000001002400000FFF8FFFFF6FE08ED00E017
:106970004FF0E02005494161054AF02182F8141DDD
:10698000002181610721016170470000DFA501003E
:106990000FE000E02DE9F047DFF8D4A0BAF80000DE
:1069A0004FF00005000635D5324C6088401C6080F1
:1069B000FBF756FDDFF8C0C0304A31489CF8007044
:1069C000677092F800800723C8262E494FF005090A
:1069D000B8F1010F22D02C4FB7F806C0BCF1000F60
:1069E00038D084F80090848944F008048481C488F5
:1069F00024F40064C480886820F004008860FD806E
:106A00001370A1F8426000204FF49661401C80B2E0
:106A10008842FBD3AAF80050BDE8F08777B1012F78
:106A200012D0C78847F40067C780886840F0040028
:106A30008860032020708CF80090E1E7878947F098
:106A4000080787810120F5E7878947F010078781CC
:106A50000220EFE7042727700C4C2570C48844F40B
:106A60000064C480886840F004008860C8E70000C3
:106A7000102C01402C070020400700203F07002079
:106A8000000C0020A4020020C80A00205D0700209E
:106A9000704700002DE9F0434FF08040018A21F05B
:106AA00001010182AA48007800287CD1A94FF87B17
:106AB000002878D1A848406C322874DCA748806848
:106AC000DFF89C924104A74DB9F804004FF0000490
:106AD00003D4401CA9F8040024E1002874D02978CC
:106AE000012611B1012912D013E14946B0F5BE7F4C
:106AF000FAD92E70CC718C71EC702C72287A0A182D
:106B0000401CC0B2147228720F28F7D301E1B9F803
:106B100002204946824201D9EE7100E0EC719048B2
:106B20008A7908300F2A15D2CB79082B0BD2C3F102
:106B30000708EB7912F800C003FA08F36344135412
:106B4000CA79521CCA71CA79082A03D18A79521C9F
:106B50008A71CC7199F80610C8460F2973D10D219E
:106B6000FBF716FAA881010A6970C0B2A87088F80C
:106B7000064098F816208A4265D198F8151081428F
:106B800061D198F80BC07849032302227748BCF101
:106B9000000F10D0BCF1010F02D0BCF1020F14D0D5
:106BA00080F86A2000E0C7E091F800C02CF00C0CDF
:106BB0000CF1080C0FE080F86A6091F800C02CF02E
:106BC0000C0C0CF1040C06E0A5E080F86A3091F89A
:106BD00000C04CF00C0C81F800C098F80C10B6EB1B
:106BE000111F04D180F86E4087F84A400EE0B2EBE6
:106BF000111F04D180F86E6087F84A6006E0B3EB9D
:106C0000111F03D180F86E2087F84A200B0717D098
:106C100001F00F01012901D0022915D080F86C6024
:106C20002C7198F80D102A7906FA02F30B406B715B
:106C3000082A41D2DFE802F00B0F4016212C333A2C
:106C400080F86C40ECE764E080F86C20E8E713B370
:106C500080F8704030E013B180F850602CE080F88C
:106C6000504029E023B180F8656087F8076123E090
:106C700080F8654087F807411EE023B187F8F940A6
:106C800080F84D4018E087F8F96080F84D6013E017
:106C900013B180F868600FE080F868400CE013B131
:106CA00080F8666008E080F8664005E013B180F87F
:106CB000676001E080F86740521CD2B22A71082A4E
:106CC000B1D398F80E108A0704D587F8F56080F8DC
:106CD000646005E0264A87F8F54080F864405481F6
:106CE000C90702D080F8294001E080F8296098F8AF
:106CF000111000F86D1FC2781E48012A1ED001B382
:106D0000012921D04FF48051A0F876101A493C2077
:106D10000870A9F80240A9F80440B9F80210491C0B
:106D2000A9F80210B9F80210B1F5FA7F04D940F2BF
:106D3000F511A9F802102C70BDE8F08344F21C7123
:106D4000E2E74FF40051DFE741F25551DCE7000084
:106D50003F070020A402002038010020001001405D
:106D6000400E0020C8060020D0040020580E00204D
:106D7000000C0020380500203C0700202DE9F05FC2
:106D8000FCF70CFD8E4D2888A5F10406C0070AD03B
:106D9000308820F008003080288820F00900288002
:106DA00002F0BAF8D9E02888DFF81892DFF81882E4
:106DB000864C80071AD5B9F8001041F00101A9F8F6
:106DC0000010B8F80000804914315030088028883D
:106DD0004FF6F95108402880308840F00400308098
:106DE000FEF71EFF84F83C00BDE8F09F2888784F2E
:106DF0004007288871D520F004002880FEF710FF96
:106E000094F83C108142EFD1308820F004003080AB
:106E1000FCF7E4FE2078410605D594F8541094F868
:106E20003B209142E0D03978400621F002013970D0
:106E300004D5FDF749FE97F82F7004E094F83C0064
:106E4000FCF7FEFC0746DFF880B140F68C2A0BF118
:106E5000180B062F47D294F83800B8423ED0384677
:106E6000FCF772FC2078C00716D094F83A0094F82A
:106E7000391000F00302914206D0A17A00F001001F
:106E800001F00101884215D1FCF710FEF9F7D2FF9D
:106E9000FCF738FF384689E0FCF708FEF9F7CAFF2F
:106EA000FCF730FF3846FCF721FE207840F0010067
:106EB000207099E7288820F008002880206B81083E
:106EC00001EBD000504515D2B8F800100844ABF8DB
:106ED0000000308840F0080003E00DE0308820F02A
:106EE0000800308080E7B9F8001041F00101A9F8EE
:106EF0000010DFE75046E7E70007288831D520F08B
:106F000008002880308820F008003080FEF788FED6
:106F100084F83C00FCF762FE387820F002003870FC
:106F20002078400604D5FDF7CFFD97F82F5004E0F8
:106F300094F83C00FCF784FC0546062D08D294F832
:106F40003800A842B5D0FCF7B1FDF9F773FF2AE08D
:106F50002048C18841F04001C180BDE8F05FFCF7E6
:106F6000B1BEC006288825D520F0100028803088C2
:106F700020F01000308097F838000C2802D2401C16
:106F800087F83800387840F002003870FDF79CFD33
:106F900097F82F50787884F8390094F83800A84290
:106FA00087D0FCF783FDFCF7ADFE2846BDE8F05F17
:106FB000FCF79CBD4EF2BE110840288014E700008B
:106FC0001004004000040040240400403801002068
:106FD00058040020000C00202DE9F04F514F85B0DF
:106FE000388820F0010038804E4800261030068096
:106FF0004D4CDFF838A14FF0010894F85C0042F6E0
:107000003029C10774D072B64948816941F40071D2
:107010008161816941F4806181614FF40040FEF734
:10702000B9FD444D00212846F9F750FC00212846BF
:10703000F9F742FCDFF800B100215846F9F73CFCB3
:1070400000213E48FBF77AFC2846F9F761FD5846D7
:10705000F9F75EFD4FF46020CDE902068DF805607A
:1070600000968DF810808DF8048069462846F9F75F
:10707000E1FD01231A460F212846F9F72CFE0121D4
:107080002846F9F719FC00204946401C80B2884286
:10709000FBD328462E600121F9F75CFE28688007A3
:1070A000FCD524484C30006894F85C1021F00101B4
:1070B0002144A1F85000F9F713FC62B6FDF710FC6B
:1070C00047F69061AAF8001094F85C00401CC0B22A
:1070D00084F85C000C2822D212491431A1F80080F7
:1070E000388840F00100388005B0BDE8F08FFFE738
:1070F000134920F00100085A12490880114945F649
:107100005800083908800F4846F65801001F0180D2
:107110000C4920200C390880AAF80090D4E70320FD
:10712000A070E1E700080040580400202C0800404F
:1071300000100240002401400028014008000240E5
:10714000E8AF0008202C01400029018802D041F05E
:10715000800101E021F080010180704710B50A88AC
:107160004B88CC881A438B8823431A430B891A43D4
:107170004B8989891A430A43A0F8442010BD002195
:10718000018041808180C18001814181818170477E
:107190000029818802D041F0010101E021F00101C4
:1071A000818070470029018802D041F0010101E08F
:1071B00021F0010101807047002930F8441F02D0FE
:1071C00041F4004101E0C1F30E010180704700006D
:1071D0004B4910B5884202D10121C41486E0B0F1B8
:1071E000804F09D0474988420DD101210220FEF786
:1071F000F3FC0021022064E001210846FEF7ECFCCC
:10720000002101205DE04049884206D1012104208F
:10721000FEF7E2FC0021042053E03C49884206D1FD
:1072200001210820FEF7D8FC0021082049E0384958
:10723000884206D101211020FEF7CEFC002110204B
:107240003FE03449884206D101212020FEF7C4FCEA
:107250000021202035E03049884202D10121441428
:1072600044E02E49884202D10121CC043EE02C4961
:10727000884202D101210C0538E02A49884202D116
:1072800001214C0532E02849884206D101214020E5
:10729000FEF7A2FC0021402013E02449884206D1D9
:1072A00001218020FEF798FC0021802009E0204980
:1072B00088420AD1841501212046FEF78DFC002169
:1072C0002046BDE81040FEF787BC1A49884202D12B
:1072D00001210C040AE01849884202D101214C0422
:1072E00004E0164988420AD101218C042046FEF7A9
:1072F0008BFC2046BDE810400021FEF785BC10BD88
:10730000002C01400004004000080040000C004038
:10731000001000400014004000340140004C0140C7
:10732000005001400054014000180040001C004083
:10733000002000400040014000440140004801405E
:10734000002A828901D00A4300E08A438281704783
:1073500030B5028C22F001020284028C8388048BF7
:1073600022F0020224F073050C882C430D8915438A
:107370004A882A43114DA8420BD0114DA84208D08B
:10738000104DA84205D0104DA84202D00F4DA84282
:107390000DD122F008054A8923F440732A4322F0D4
:1073A00004058A882A438D891D43CB892B4383801A
:1073B0000483C9888186028430BD0000002C01400E
:1073C00000340140004001400044014000480140B9
:1073D000028B22F008020A430283704770B5028CC8
:1073E00022F010020284028C8488038B0D8823F41F
:1073F000E6464FF6FF7303EA052535430E8922F072
:10740000200203EA061616434A8803EA02123243B0
:10741000104EB04202D0104EB04215D122F080067C
:107420004A8924F4406403EA0212324322F04006FF
:107430008A8803EA021232438E8903EA86062643CB
:10744000CC8903EA8404344384800583C988018796
:10745000028470BD002C014000340140028B4FF6C5
:10746000FF7322F4006203EA012111430183704794
:1074700070B5028C22F480720284028C8488838B23
:107480000D8823F073031D4322F400730E894FF619
:10749000FF7202EA06261E434B8802EA03233343A7
:1074A000104EB04202D0104EB04215D123F4006607
:1074B0004B8924F4405402EA0323334323F48066C7
:1074C0008B8802EA032333438E8902EA0616264399
:1074D000CC8902EA0414344384808583C988818777
:1074E000038470BD002C014000340140828B22F0E7
:1074F00008020A438283704770B5028C22F48052DE
:107500000284048C8288838B0D8823F4E6464FF630
:10751000FF7303EA0525354324F400560C8903EA7A
:10752000043434434E8803EA06362643094CA0420D
:1075300002D0094CA04205D122F480448A8903EA92
:107540008212224382808583C988A0F84010068475
:1075500070BD0000002C014000340140828B4FF6CA
:10756000FF7322F4006203EA012111438183704713
:10757000018582827047828822F070028280828830
:107580000A4382807047A0F84010704730B50288E7
:107590001B4B1C4C98420DD0A0420BD0B0F1804F39
:1075A00008D0194DA84205D0184DA84202D0184D58
:1075B000A84203D122F070054A882A43154DA842FB
:1075C00006D0154DA84203D022F44075CA882A433C
:1075D00002808A8882850A88028598420AD0A04261
:1075E00008D00E4A904205D00D4A904202D00D4A72
:1075F000904201D1097A01860121818230BD0000CB
:10760000002C01400034014000040040000800400C
:10761000000C0040001000400014004000400140F9
:1076200000440140004801404FF6FF718180002175
:107630000180C1804180017270470029018802D019
:1076400041F0020101E021F00201018070470029B0
:10765000018802D041F0040101E021F00401018021
:10766000704780092830FF2801D9FF207047C0B239
:1076700070472DE9F041B1F9025000231E240F227A
:10768000854203DDB1F90000BDE8F081B1F97A501F
:10769000854202DAB1F97800F6E701EB8205B5F927
:1076A0000250854201DA134600E01446E2185208FF
:1076B0005D1CAA42F1D101EB8203B3F9024084427E
:1076C00006DAB3F9067031F92250B3F9046005E027
:1076D00033F9027C31F9225033F9046C001BC117D5
:1076E00089013A1B41EA9061D3178001F8F71AFD2E
:1076F000721BA0FB024601FB0261D31700FB0310C3
:10770000810641EA9410284400B2BDE72DE9F04F0C
:10771000DFF8B8B16A48DFF8AC91DFF8ACA190F8B7
:107720000EC0BBF91A70BBF91C60BBF91850BBF94D
:107730006C10BCF1070F48D2DFE80CF08D041A3052
:10774000485E7600D9F80020C284DAF8002002856D
:10775000C28C038DA7EB820212B2A6EB83034A43CD
:107760001BB2594342F3CF2241F3CF23D11870E02B
:10777000D9F800208284DAF800200285828CA5EBFB
:10778000820213B2028D4B43A6EB820212B243F384
:10779000CF24514341F3CF23E11814E0D9F800205E
:1077A0000285DAF800208284028D838CA6EB8202A7
:1077B00012B2A5EB83031CB24A43614342F3CF23C9
:1077C00041F3CF24191949420AB244E0D9F8002004
:1077D000C284DAF800208284C28C838CA7EB8202F8
:1077E00012B2A5EB83034A431BB2594342F3CF22A3
:1077F00041F3CF24111914E0D9F800208284DAF87B
:107800000020C284828CC38CA5EB820212B2A7EB4B
:1078100083034A431BB242F3CF24594341F3CF229F
:10782000A11849420BB216E0D9F800200285DAF817
:107830000020C284028DC38CA6EB820212B2A7EB99
:1078400083031CB24A4342F3CF23614341F3CF2267
:10785000991849420CB2BBF91E50594605F21E5602
:10786000A64201DACE8306E0A5F21E55A54201DD4F
:10787000CD8300E0CC83B1F9204004F21E5595423F
:1078800001DA0D8406E0A4F21E54944201DD0C845A
:1078900000E00A84B1F9222002F21E549C4202DA6E
:1078A000ABF8224008E0A2F21E529A4202DDABF889
:1078B000222001E0ABF82230417B8173BDE8F08FDC
:1078C000A40200203C2401403C280140380500204F
:1078D0002DE9F04704467048714E002702786F4842
:1078E000022AB0F9341004D0082A6ED0092A6DD0CB
:1078F000CDE0C27B022A02D1B0F844205AB1A4F8EC
:10790000421071810423B6F908101A460020FEF7D0
:107910001DFF3081BBE06349DFF88C81496A0D149B
:10792000E58090F84A1099B10089DFF88091C0F3A2
:10793000C001C0F30020814223D1D8F8440040F2B6
:10794000BA41884240DD40F66A1188420ADC15E0FF
:10795000B4F9020040F2DA21884279DD40F26A414E
:10796000884204DD0823B4F942101A464EE0A0F222
:10797000DA20F8F760FD00224D4B56E0A0F2BA4045
:107980004FE04C480078C0060CD5D8F8440041F2CE
:10799000243188425CDD41F2D4718842E2DC00F699
:1079A000DC4020E04448DFF8149190F87010012981
:1079B0000DD090F86F00012809D041480178C9071F
:1079C00046D04049098889B142E05AE05DE0B4F907
:1079D000020041F6DC6188423ADD42F2341188420D
:1079E00010DC00F59270A0F500501AE0B0F910001C
:1079F000B4F90210A0F59672914229DD00F5967255
:107A000091420BDDB4F9421020231A460020FEF704
:107A10009DFEA4F84200002817DB1BE0081A00F5C1
:107A20009670F8F708FD00224B46F8F770FC0E221E
:107A3000F8F7DCFCF8F736FD00B2C0F5804068438B
:107A40008013A4F84200002D04DCA4F8427001E089
:107A5000A4F842501C48B0F91210D8F85000081A87
:107A6000718B01EB600000B2F082002800DCF7822D
:107A7000B4F94200B6F91610884200DB084670815E
:107A800004E01248B0F87C00F9E77181378184F88E
:107A90004070BDE8F08700003F070020A4020020EE
:107AA0004C000020380500203801002000C0924022
:107AB0000000794010070020580E002000C08240CE
:107AC000B00A002008000020C80A0020140C002082
:107AD0002DE9F041B1F9025000232B2415228542F3
:107AE00003DAB1F90000BDE8F081B1F9AE5085428A
:107AF00002DDB1F9AC00F6E701EB8205B5F9025001
:107B0000854201DD134600E01446E21852085D1C70
:107B1000AA42F1D101EB8205B5F90230834206DABF
:107B200035F9026C35F9044C31F9221006E01E4695
:107B300031F92240B5F90630B5F90410801B091B54
:107B4000C5178911AD0345EA90458703A1FB070CD2
:107B5000CA1702FB07C201FB05219A1BD317F8F7CE
:107B6000E1FA000A40EA0160001900B2B0F5804F66
:107B7000B9DB43F6FF70B6E770B5134C40F224450D
:107B80002946204600F02CF800281BD0204600F0A3
:107B900046F82946204600F01DF80C4C00212046EE
:107BA000FAF7CCFE2046FAF747FFC0F16400084917
:107BB000C0B20428087201D900F0AEF9BDE87040E7
:107BC000FAF778BF70BD000000380140580002404D
:107BD000740600200A0A01219140C94301807047C0
:107BE00030B501F01F0201240025C1F3421304FA4D
:107BF00002F2012B0FD0022B0FD0838A4FEA112102
:107C00000088134204FA01F400EA040001D000B134
:107C10000125284630BD8389F0E7038AEEE7808896
:107C2000C0F308007047000070B5214C2068214D5A
:107C3000400103D520492846F9F746FA206800019B
:107C400004D51D492846FF31F9F73EFA2068C000E7
:107C500003D51A492846F9F737FA1948194A01781D
:107C6000CB0712D192F82F30012B0ED0FAF75EF924
:107C70002068C0F382611448072916D0216811F0EA
:107C8000E05F01D15521017070BD012382F82F30D2
:107C900021F0010101700D4801680D4A01F4E06115
:107CA00011430160BFF34F8FFEE70021EBE70000B7
:107CB0000864004000640040010000380000013802
:107CC0003E080020CC0E0020480800200CED00E00B
:107CD0000400FA05F0B585B0042000258DF80800F1
:107CE0000702844C009501958DF80A508DF81350C9
:107CF00039462046F9F748FB01281DD17E4E06F88B
:107D0000305FF9F75FF9206840F40040206079485F
:107D10001430016821F001010160784D286800F0FD
:107D2000FBFD002176A001F051FE28603946204677
:107D3000F9F7E2F90120307002212046F9F724FB1F
:107D400001287CD16A4600212046F9F7F3FB01980F
:107D50006E4920F0604088609DF80A1008291BD108
:107D60006B4908440C2817D2DFE800F0060BBDBDB4
:107D7000BDBDBD1752717CA364489DF80B106F30D8
:107D80009BE0624A0020694617320B18DB7A1354D5
:107D9000401CC0B20828F8D3A5E05C499DF80B0050
:107DA0004F3103090A7860F3030263F304124309B5
:107DB00063F34512800960F387120A709DF80C0086
:107DC00048709DF80D0088709DF80E00C8709DF8F1
:107DD0000F000A7960F30002400860F347020A715D
:107DE0009DF8100048719DF811208879930862F37E
:107DF000010063F38300120962F3071088719DF894
:107E00001220C87962F30600D20962F3C7104EE06F
:107E100040489DF80B1001709DF80C1041709DF8C2
:107E20000D1001F003028270C1709DF80E100171F7
:107E30009DF80F1041719DF81010817100E056E01F
:107E40009DF81110C1719DF8121001724BE02F487E
:107E50009DF80B205730017862F30101920862F31C
:107E600087012AE029499DF80B205F31087862F3E9
:107E70000300120962F3071008709DF80C004870A7
:107E80009DF80D20887862F30600D20962F3C710CE
:107E900088709DF80E00C8709DF80F0008719DF85D
:107EA000100048719DF8110088719DF81200C8718A
:107EB00019E016489DF80B10673001709DF80C1002
:107EC00041709DF80D1081709DF80E10C1709DF8E5
:107ED0000F1001719DF8101041719DF81110817102
:107EE0009DF81210C17102212046F9F705F905B07D
:107EF000F0BD000000640040CC0E00204C080020C3
:107F00006465765F63616E310000000060070020E9
:107F1000FFFE00E71010002070B51D4D00242878EA
:107F2000432834D16878462831D1A878502807D022
:107F3000512805D0812803D0892801D0212826D1B5
:107F4000144E7071E9787172A81C891CFAF758F800
:107F5000B072717A294409793182884217D106F1C9
:107F60000E00017841F0020101700B48016841F0F8
:107F700020010160317A0948002204E02B5D03559D
:107F80002A55641CE4B28C42F8D38078707170BDBD
:107F9000F0080020740600200C0C0140920D002017
:107FA00070B51D20FDF7C8FAFCF78EFD1D20FDF70A
:107FB000D9FA154890F82F10144D0623144C85F863
:107FC000381090F83B1095F83B201143012A04D05B
:107FD000022A07D0042A0AD010E0827A8A420DD001
:107FE000007B09E0027D8A4208D0807D04E0827F28
:107FF0008A4203D090F82000884200D123700020EC
:1080000085F8400070BD00005804002038010020B1
:108010003F0700200B4800214180A0F1B8018A8968
:108020008280CB891A44C2800B8A1A4402814B8A0F
:108030001A444281898A1144818143F6FF71C181CA
:1080400070470000F0010020084940F61C72B1F9A9
:108050000C00904202DA00F59F7005E041F2E30265
:10806000904201DDA0F59F70C88170474C00002050
:1080700038B51348C16941F00401C1611E208DF873
:10808000000002208DF801008DF8020001248DF817
:1080900003406846FDF772FA0A49842008800949BE
:1080A00047F690602C3108800020091F08800549A0
:1080B00014310C80091F0880081F048038BD00009F
:1080C000001002400008004030B420491E4A4578A4
:1080D0008B7A114692F83B4091F83910AC4218D196
:1080E0004BB10379994202D04379994201D1407949
:1080F0001AE0807909E08379994202D0C479A142DB
:1081000002D182F82F3011E0407982F82F0030BC84
:108110007047C578AC42FAD16BB1C379994202D0AD
:10812000037A994205D1007A82F82F0030BCFEF71D
:10813000BFBB407AE9E7437A9942E2D00479A14291
:10814000DFD0007AE1E70000580400203801002069
:10815000FEE700002DE9F0470446007F012868D1C2
:108160003548E1880288511A89B2072916D3008858
:10817000E080B4F9000044F2DD414843401346F684
:10818000D96148438013A060401000B2A0814FF035
:108190008051B1FBF0F0F8F749F92061B4F90C60B7
:1081A00096B1B4F902104DF6B05048430014A082C5
:1081B000B4F904704DF6B05207FB02F24FEA2245C3
:1081C000E58204D4024603E00020E08330E042422E
:1081D00012B22283002D01DB2B4600E06B421BB262
:1081E000DFF85890638398464FF4804AB24208DA29
:1081F000F8F713F92169F7F7E6FFF8F73AF9801372
:1082000004E0002901DA484600E05046E083B0452A
:1082100009DA2846F8F701F92169F7F7D4FFF8F7EA
:1082200028F9801304E0002F01DA484600E05046A8
:108230002084BDE8F08700004807002000C0FFFF51
:108240002DE9F0414C484D4E00250078A6F1500430
:10825000022806D14A4FF87B022802D1B7F8440021
:1082600030B1A5862564B56284F83850BDE8F08148
:1082700044488168C068494300FB0010FBF766F979
:1082800040F233314843810BB4F8440043F6CC420A
:10829000504301EB903080B243F69911A4F84400AA
:1082A000884209D338481146B0F90400884203DBFC
:1082B00097F84A00032813D00123B4F934101A4662
:1082C0000020FEF743FAA086B4F84000012301B273
:1082D0001A460020FEF73AFA20648003B06226E0D6
:1082E000B4F8460041F69A13A0F51852663A9A423D
:1082F00009D2B4F94400214AFAF7C8FF20640120EA
:1083000084F8380022E044F24711884212D994F8E8
:108310003800D8B11D480178491CC9B20170022942
:1083200014D30570206C10B1401E206408E084F85E
:1083300038500BE0A0F58040B0F5A47F03D2206C4C
:108340008003B06202E084F83850B562B4F84000AF
:108350000A4980B20839323401F006FDB4F9000050
:10836000B4F91810414389136180B4F916104843D9
:108370008013A0807AE700003F070020800A0020D9
:10838000A4020020BC090020E205002032010020E8
:108390000D480021A32280F82810C1838186503027
:1083A000C2600E22028241F262024261082202830E
:1083B000418341F2555282839203C0E9081240F290
:1083C0008E32826081627047300A00202DE9F041D0
:1083D0000546FBF7B3F9204C204E0746206861683C
:1083E000421C8A4220D009B93F281DD004EB00105E
:1083F000AA7A05F10B010E30F7F7C5FE216868680F
:1084000004EB011188602168A87A04EB01118881CE
:1084100072B62068401C2060402801D300202060F4
:1084200062B6307888B114E03846FBF76FF90A2855
:10843000D4D3706800F070FA002109A001F0C6FAE8
:1084400070604FF0FF30BDE8F08155203070F9F7D3
:108450006DFD0020F7E70000A81400204808002068
:108460006465765F63616E310000000010B5040042
:108470000B462D4AC3F1000028D56442002B12DAC6
:10848000A04207DA214600F0F1FB32F81000C0F5F7
:10849000404041E00146204600F0E8FB32F8100081
:1084A00000F5004038E0A34208DA2146184600F003
:1084B000DDFB32F8100000F540402DE0204600F0D2
:1084C000D5FB32F81000C0F5803025E0002B12DA21
:1084D000A04207DA214600F0C9FB32F8100000F58F
:1084E000804019E00146204600F0C0FB32F8100041
:1084F000C0F5004010E0A34208DA2146184600F01B
:10850000B5FB32F81000C0F5804005E053B12046BD
:1085100000F0ACFB32F81000B0F5004F01DDA0F523
:10852000803010BD002010BDF4AF00084043801320
:10853000494300EBA13000220302002B14DDB3F508
:10854000001F01DC802001E04FF4005093FBF0F1AC
:10855000014401EBD1714910814206D0521CD2B2C4
:108560000846062AF2D300E00021C80000B2704796
:1085700002E008C8121F08C1002AFAD170477047EC
:10858000002001E001C1121F002AFBD1704700004A
:108590002DE9F047BD4CBE4821880288511A89B2A6
:1085A0000F297DD30088A4F13C052080288F08B1D5
:1085B000401E28872B78B74AC3F3810001281ED0BC
:1085C000022821D0118BB148B44EDFF8CC92407E06
:1085D000B6F806C00027B1F5926F1CD8142818D33E
:1085E000782060764CF01000F08040F26660A88140
:1085F00023F001002870D77389F8007018E0108B01
:1086000000EB4000C00302E0108BA5494843010C79
:10861000D9E7401C04E0B1F5216F09D910B1401E23
:10862000607605E02CF01000F08043F00100287027
:10863000B5F90200B5F914304143C3EBC303C1F3EC
:108640008F31C3F3D10303EB510109B2A9829046E4
:10865000128B4FF080535043B5F91620C0F38F3082
:10866000C2EBC202C2F3D10202EB500000B2E882B8
:10867000AA6A42431213EA6293FBF2F22A63894A1E
:108680001080A2680A44A260E1680144E160207C95
:10869000401CC0B22074072802D942F3CF0000E08A
:1086A000E8E02883C9106983E760A76041F6C80144
:1086B0002774884204DD2A8B7B49B1FBF2F1E98102
:1086C000C117890341EA9041800342F69B4200238F
:1086D000F7F728FDA8846D482A78A0F13C0093079D
:1086E000B0F90600C2F3810200EB801101EB00310A
:1086F00041F30F3115D5012A07D0022A0BD04EF6CF
:10870000AC3141430914A18011E049F25862504351
:108710000014A08020E04CF20C3141430914A180E8
:1087200026E0012A0ED0022A18D0A08069845F4971
:1087300048430014A4F81E00FAF73EFB5C4800888A
:10874000C0B143E04AF2904242431214A2804BF27D
:10875000C822504300146884E183EDE74CF634519D
:1087600041430914A1804DF66C31414309146984D9
:108770005049DDE795F8200000BB88F80F7089F8B4
:108780000070B5F91A00A0F514512C39B1F56E7FBF
:1087900018D2617FF42912D94749E880434AA1F8E9
:1087A000460050430014A880A1F84400FF2085F83B
:1087B000200081F8280041493C20087006E0491C4F
:1087C000617703E0607F08B1401E6077B5F91A0059
:1087D000B4F91E203A4990420DDDA27E7D2A08D9C7
:1087E000F28842F00802F2800A7822F002020A704F
:1087F0000EE0521C06E0A2F23D12904208DAA27E80
:1088000012B1521EA27603E0F28822F00802F28032
:10881000B4F90420904214DA2A4B9B68B3F5FA7F2E
:108820000FDAE07E3E2809D9F08840F01000F08091
:108830002777087820F0020008700CE0401CE076F2
:1088400009E002F23D12904201DD8888A0B1207F4C
:1088500008B1401E2077B5F91810606908446061BE
:10886000217E491CC9B221761F2903D94011A88352
:1088700067612776BDE8F087207F7D2804D9F088DE
:1088800020F01000F080E6E7401CE3E70C05002034
:1088900048070020A40200203F070020000C002011
:1088A00030330100700B002074E8260B188601009D
:1088B0004A070020E0380100580E00203C07002045
:1088C000E205002038050020024941F2F460886288
:1088D00070470000D004002070B50D4C207828B1FE
:1088E000012808D0062505280FD10BE00948F9F723
:1088F00097FD012004E00748801DF9F791FD052050
:10890000207070BDF9F7ACFD2570257070BD0000BA
:1089100040070020FCAE00080A4A4FF0FF31B0EBE0
:10892000A20F0CDA00280ADB0749096851F8200079
:108930004068006900B100476FF0050070470846C5
:1089400070470000040000007C08002070B50A4D4C
:10895000A86870B100240948AC60F8F75DFC0848CD
:1089600004604460A0F58160046044602C700020C5
:1089700070BD6FF0040070BD480800200064004026
:10898000A81400207FB505460024631E244A4FF03A
:108990000050072D41D2DFE805F04004111E2140B0
:1089A0003C00814208D2D068202805DA1D4B43F8EC
:1089B0002010401CD0600CE01C4627E08142FBD216
:1089C00010692028F8DA174B803343F82010401C38
:1089D00010610023F0E7F8F735FC17E000208DF870
:1089E0000B000121ADF800000422ADF80400ADF841
:1089F00008008DF80C108DF80A00ADF80220ADF8D3
:108A000006208DF80D106846F8F758FC204604B093
:108A100070BDBDE87F40FAF725BF1846F7E70000B4
:108A200048080020B0180020F8B5414EB068012871
:108A30007BD04048F8F7F0FB01210820FDF7D8F87B
:108A400001210846FDF7D4F801214806FDF7B8F8E2
:108A500001214FF4EA10FAF71DFE4FF48070ADF8D3
:108A6000000003248DF802400420334D8DF80300EC
:108A700069462846FAF7BCFD6815ADF800008DF888
:108A8000024018208DF8030069462846FAF7B0FD29
:108A900014208DF8000002278DF8017000248DF855
:108AA000024001258DF803506846FCF767FD13204E
:108AB0008DF800008DF801708DF802508DF803508C
:108AC0006846FCF75BFD16208DF800008DF801402C
:108AD0008DF802408DF803506846FCF74FFD1749AA
:108AE0000120FFF74FFF16490120FFF74BFF154903
:108AF0000120FFF747FF14490120FFF743FF134907
:108B00000120FFF73FFF00210320FFF73BFFF8F7AD
:108B10002FFB0F4804604460A0F58160046044604E
:108B200034700020B560F8BDFFE74FF0FF30FAE782
:108B30004808002000640040000C014020FF40185D
:108B400020FF431820FF441820FF451820FF251858
:108B5000A81400202DE9F04781461E4886B017462C
:108B600080680E46A0B14FF0FF381FB36846FAF791
:108B700087FE401C0ED00DF10B019DF80A208A469D
:108B80004846019DF7F7FFFA9DF80A403D601DE059
:108B90006FF0040006B0BDE8F08700BFFAF762FE90
:108BA000411C15D0A84213D16846FAF769FE019816
:108BB000A84201D04046EDE79DF80A2009EB0400E9
:108BC0005146F7F7E0FA9DF80A000444B442E5D3B1
:108BD0002046DFE7480800202DE9F04706462248F6
:108BE00086B00024806888B1601E002A10D0126808
:108BF0000192B2F1005F0BD2CF0801F007054FF0F0
:108C000000084FF004094FF0080A17E06FF0040065
:108C100006B0BDE8F08700BF8DF80AA08DF8089077
:108C200006EBC4008DF809800168CDF80B10406890
:108C3000CDF80F006846FFF7C9FB641CBC42EBDBB4
:108C40007DB18DF80A508DF808908DF8098006EBFB
:108C5000C4012A460DF10B00F7F795FA6846FFF7B5
:108C6000B5FB0020D4E7000048080020090A05D021
:108C7000B0FBF1F0FF2800D9FF20704700207047BB
:108C8000D0E90021C368521A5A4301EBA231816036
:108C900041607047B0F90020B0F90210B0F9063019
:108CA000521A5A4301EBA231818041807047000083
:108CB00030B5494B188849498A89801A85B2484895
:108CC000484A0F2D047801F14C001DD31D888D8179
:108CD000117A090713D5022C01D0434912E0434D04
:108CE000B0F90210B5F90050A94205DC02DA01F131
:108CF000020108E0458007E0A1F1020103E0022C37
:108D000002D13B4909884180B0F840101D88691A9A
:108D100089B29C2949D31988A0F84010D16A002350
:108D2000B1F5804F31DB3349096DB1F5405F2CDD82
:108D3000314940F26665B1F91010A94212DD43F6DF
:108D40009915A94202DB40F2333108E040F2333595
:108D5000A1F26661694343F2333591FBF5F1A0F866
:108D6000441001E0A0F844302449B2F80A510978CF
:108D7000C1F381012DB100BFB0F8441001F21E51C2
:108D80001CE092F84A20032A10D0A0F84430022CAC
:108D900001D0A0F84430B0F95C10B0F9443001F1D2
:108DA00014029A420DDAA0F85C2030BD012901D0EE
:108DB0000229E1D1B0F8441001F23331A0F8441097
:108DC000E5E703F11402914203DD1439A0F85C10C9
:108DD00030BDA0F85C3030BD480700200000002006
:108DE0003F070020A4020020CE040020CC04002075
:108DF000C80400203801002038050020D0040020DD
:108E00002DE9FC4101210220FCF7DAFE01211920A5
:108E1000FCF7EEFE01213C48FAF73CFC4027ADF898
:108E2000007003248DF802400420384D8DF80300B3
:108E300069462846FAF7DCFBE001ADF800008DF842
:108E400002401C208DF8030069462846FAF7D0FB43
:108E50004FF4E0712846FAF752FCA815ADF800006F
:108E60008DF8024010208DF8030069462848FAF773
:108E7000BFFB4FF4A060FCF7B3FB1D208DF804008E
:108E800001268DF8056000258DF806508DF80760E5
:108E900001A8FCF773FB1F498C2008801D494FF681
:108EA000FA702C3108806E20091F08801948143090
:108EB0000680184808300780164920310D80154A71
:108EC000D020121D1080134A45F2F3001832108092
:108ED0000A1F45F2500010800E4A4FF6FF703832DC
:108EE0001080121D1080121D108041F21B1008808E
:108EF00000F012F8FAF7E6FE064810300580001F71
:108F00000480BDE8FC810000000C1A000010014044
:108F1000000C01400004004070B51D20FCF701FB6F
:108F20002A4D40212846FAF7E1FB8400802128469B
:108F3000FAF7DCFB44EA4004A9152846FAF7D6FB09
:108F40000443E0B2224C84F83C00FAF779FC054671
:108F5000052805D91F48C18841F04001C18001E0C2
:108F600084F838501C48007A000703D594F838007C
:108F70001A490D5C4FF6FA702063E062A0626062ED
:108F80002062E061A0611648606300206064206593
:108F900084F83F0084F84000FAF700FCA07AFF282C
:108FA00011D0022084F83D000E480088A0662846B3
:108FB000FBF7EAF8207820F001002070BDE870404F
:108FC0001D20FCF7C4BA0120ECE7000000100140AE
:108FD00038010020000C0020A4020020F0B8000896
:108FE000DCFF0500240400402DE9F0434D484E49C4
:108FF00002880B889A1A92B20F2A67D309880180D7
:109000004A49C98B027D00EB42029180017D491CD7
:10901000C9B20175082959D3002404752246017D7F
:1090200000EB4103491CB3F90430C9B202EB6302FF
:1090300012B201750829F2D33D4904753D4B4A80AF
:1090400044800E789D895FEAC67C40F638694FF00F
:10905000030714D0A2F22B5C42F6E858C44520D393
:10906000A1F1020C26F00204ACF8002047750C7048
:1090700040F22B54A24211DA45F004021EE046F001
:1090800001060E704A4507DD45F001029A8126F07F
:1090900002020A70477517E0447515E045F00202B8
:1090A0000CE04A450CDA8775427D12B1521E4275BA
:1090B0000AE046F002020A7025F007029A8103E0F6
:1090C000837D2BB15B1E837540888880BDE8F0836B
:1090D00042F6AA239A4222DAB1F904302BB941F2BE
:1090E000CD05AA4201DA4480EEE7134C920302EB6D
:1090F000843241F67244B2FBF4F214B24FF480555C
:1091000002464480AC4200DA5580B2F90240E41ACB
:1091100004F5A374B4F5237FD6D84380D4E74FF485
:109120008043FAE7940C002048070020A4020020A6
:10913000E2050020000C0020C8F1FFFF2DE9F041FE
:109140006D4CDFF8B8E14FF0000594F83410C80713
:1091500006D094F938104B42002958DD0E4657E0EE
:10916000674884F83750A4F84250664A90F83800AF
:1091700084F840009586CEF80450CEF80850624E30
:1091800040F26663CEF80C50A4F87C3036F810003C
:109190005E4E768830444FF6FF7606EA800024F86B
:1091A000300B4FF0806044F8040CA32020846084CE
:1091B0005810A084E38440F69910208558006085FB
:1091C0004FF48050A08541F23330E08541F2666073
:1091D000208641F69910608641F6CC40A0864FF477
:1091E0000050E08642F23330208742F266606087AA
:1091F00042F69910A08742F6CC40E08782F8A15051
:1092000041F00100207184F84450BDE8F0811E4611
:1092100094F937004242002801DD074600E0174676
:10922000F61B012E0BD0002800DB02465FFA82F607
:1092300084F8380094F84F00012805D041E0002957
:1092400000DA1946CEB2F3E794F939305942002BCF
:1092500001DB184600E0084694F93A20C7B25042B4
:10926000002A01DB944600E08446BC4508DD002A64
:1092700000DA0246D7B2002B00DA0B46D8B207E07C
:10928000002B00DA0B46DFB2002A00DB1046C0B22A
:1092900004EB4000B0F9501004EB470030F9502FB8
:1092A00011444910018084F84F5084F83E5084F8EE
:1092B0003D5084F83C5084F83B5084F83A5084F890
:1092C000395004EB46007546B0F9500024F8420FBF
:1092D000BEF80410C82309B26422FDF737FA6860AB
:1092E000E968401AA9680844A860B5F90010484325
:1092F000C013E860608788E7140C0020D0050020C8
:1093000038010020A402002002B900084C0000200F
:10931000F0B4544890F83410C90776D0524990F808
:109320004030002291F838108B426FD04F4CA0F89B
:1093300072204F4DE65C04468E4294F9374002D0CD
:10934000EE5C8E420FD1641C64B280F83740EB5C57
:109350008B4202D1641C80F8374090F937300F2BD4
:109360001BDD0F2317E0434DEE5C434D8E4202D0D0
:10937000EE5C8E4211D1641E64B280F83740EB5C23
:109380008B4202D1641E80F8374090F937406FF06D
:109390000E039C4201DA80F83730324B90F83F5090
:1093A000393390F83740EC5490F83F305B1CDBB217
:1093B00080F83F30062B01D380F83F2090F93940E8
:1093C00090F93B309C420ED190F93D40A3420AD126
:1093D00090F93A4090F93C309C4204D190F93E40DB
:1093E000A34200D1012280F84F201F4A80F840108C
:1093F00090F937501378214A012D0DDD14465E0790
:10940000A46804D544F0080403E028E015E024F043
:109410000804946080F83510B5F1FF3F0ADA5B0765
:10942000936802D523F0080301E043F0080393603A
:1094300080F83510F0BCFAF7B1B990F84F10012957
:109440000DD1B0F8721043F60953491C89B2A0F847
:109450007210994203D9A0F8722080F84F20F0BC16
:1094600070470000140C002038010020E4B8000808
:10947000EAB80008F6B80008FCB80008A40200200A
:1094800010B502884188B0F90830114409B281FB57
:109490000313890B428041EA8341B0F90420B0F9FB
:1094A000063082FB0332940444EA933211448180F3
:1094B00010BD000030B52049204AB1F86A3010884C
:1094C000C01A80B20F2836D31088A1F86A001C4D4C
:1094D00000204FF000432A5C940903D00124B4EB30
:1094E000921F24D1D20622D0164A52F820201268A8
:1094F000134C123434F81040224201EB000494F96A
:10950000722008D00A2A04DB0A6823FA00F42243F6
:1095100008E0521C09E012F10A0F05DC0A6823FA80
:1095200000F4A2430A6002E0521E84F87220401C3C
:10953000C0B21128CFD330BDE80500204807002075
:10954000F8B30008F8B400082DE9F0077A497B4821
:109550000A8903889A1A92B2082A75D3008808816A
:10956000A1F12C0042890AB1521E4281744A92F83C
:109570002820802A68D302F03F020A70C2890AB10B
:10958000521EC281B1F90620902A0CDB8A46FF2ABE
:1095900009D08146C089002856D16A480023007846
:1095A000092805D005E0BDE8F007634800F0C0B920
:1095B0000823654A92F8EE500DB143F00403634866
:1095C000817AC90701D043F00203D2F808C05FEAEC
:1095D0000C5101D543F00103176800215C4EFC03D8
:1095E00002D596F8654004B18021C4885FEA4468DA
:1095F00001D541F040015FEA845801D541F02001D6
:109600005FEAC47801D041F01001007A400701D52B
:1096100041F008014F480078C00701D041F0040133
:10962000A00601D541F001010020012D00D1082044
:1096300096F870508DB992F84A20032A05D0022A74
:1096400006D0012A07D008E072E040F0030004E0F1
:1096500040F0020001E040F001007A0701D440F040
:109660002000CCF3C0020025CCF3002C624502D1CF
:109670003A0700D4042596F86F20012A01D145F05D
:109680000105354A0027BC4612783E46C2F38102E6
:10969000012A04D0022A04D0032A04D004E00226BE
:1096A00002E0042600E010262C4A64060ED5224C67
:1096B0001C342478240609D51478640606D4284A74
:1096C00040F6CC44926D6243140C05E0B2F8B6202B
:1096D00040F699146243940B4FF008088AF80A8008
:1096E0004FF061088AF80B808AF80C308AF80D1068
:1096F0008AF80E008AF80F508AF81070270A4B403B
:1097000083F06901414069408AF8117079408AF814
:109710001240614052468AF813C071408AF81460C2
:1097200051754FF4C871A9F80E10FF20AAF8060071
:10973000BDE8F00770470000F4060020480700204D
:10974000E80500203F070020A4020020000C0020B4
:10975000580E0020B00A0020D0040020380100205C
:10976000540900205D48816941F0FC0181614FF49A
:10977000A060FBF735FFFAF733FBF7F721FAFBF7A9
:10978000AFFD002156A000F021F958490860FDF70F
:10979000EFF8FCF7E1FEFFF733FBFBF70DFAFFF7FD
:1097A000BBFBFAF78FFA524D4FF40050A5F81A019F
:1097B000FCF7C6F8FCF77AF800214FF4FA5340F2B0
:1097C000EE220020401C80B29842FBD3491C89B293
:1097D0009142F6D3474C002684F87260F7F780F880
:1097E000F8F714FF42F21C202083401C608342F2F1
:1097F0000320A08342F2AA00A080F8F70DFCFEF738
:1098000037FC10223C493D48F6F7BDFC01F0F6F963
:109810003B4C3D4FE08820F04000E0803948017823
:1098200021F020010170FA20F8814FF49670A5F81C
:109830004200FFF749F835493548FBF7E2FF354864
:10984000FCF704F83448416A88473448416B88473C
:10985000FEF79EFD3248F9F7ABFAF8F70FFC3149F5
:109860004220C8803049C8603048F7F755FBA868E7
:1098700020F48070A8603E71E088E0812089208219
:1098800060896082F9F716FEF9F772FDFEF780FE37
:1098900001F034F9FFF7A8FB00F034FAFFF70AFEF5
:1098A00000F0E4FFF9F758FBF8F712FCFAF78AFC2E
:1098B000FFF7FEF9FCF72CFAFAF7ACF8FAF7DEF846
:1098C00000F0B2F8FFF740FE1548F9F71DF900F077
:1098D000A5FAFCF785FEF9F7A1FACDE700100240E2
:1098E0006465765F63616E31000000004C08002003
:1098F000A402002038050020580E00202806002071
:10990000000C0020380100203C070020000A002045
:10991000D00900200C04002020000020CC000020F2
:109920003C0B00203007002040040020B00B00203A
:10993000F0B523490278B0F9064000231F4E31F8F4
:109940001210FF2C18D0B0F904701E4DBC4231DA51
:1099500000EBE40704F00704BF7AA7408478FFB265
:109960003CB190F801C0ACF1010C64451FDA3C0633
:109970001DD455F822200DE056F82220116012491E
:109980008A79521CD2B28A71022A02D38370C380B0
:109990008B71F0BD11608178491CC9B28170427829
:1099A0009142F6D38370C188491CC180F0BD56F83E
:1099B0002220EFE755F822201160F4E7D8B500081F
:1099C0000AB4000880B50008C80600202DE9F0415F
:1099D0000F4680460024124D124E08E0286850F8C9
:1099E000240001684046F6F7E0FB38B1641CB4EB94
:1099F000A60FF3DB6FF00100BDE8F081286850F896
:109A000024004068016829B13846884728B16FF0C2
:109A10000200F1E76FF00500EEE72046ECE70000FA
:109A20007C08002004000000F0B561486149B0F8EE
:109A30006C200B889A1A92B29C2A7BD30988A0F8D2
:109A40006C105D495D4F91F82A1001F0070297F8FC
:109A50004A10022A00D1491E594C80F83E104FF09E
:109A60000203E2884FF00001550401D5012236E0DF
:109A7000A489E50601D5062231E0250701D5082293
:109A80002DE0550603D44F4D2D78AD0601D50422A7
:109A900025E0150501D5072221E0150601D50A228A
:109AA0001DE0950601D50C2219E0150701D50B2202
:109AB00015E0550701D4D50501D510220FE0D506D4
:109AC00001D505220BE0650703D4A50701D4E407FF
:109AD00002D080F86E3007E0920403D5032280F8AC
:109AE0006E2001E080F86E10374A384C92F820E082
:109AF000324A251FD2F808C02D4AB2F87060721C95
:109B000092B2BEF1000F0DD02CF4000CC7F808C0C3
:109B100090F86E70B7B11E2F1AD090F86F200AB36C
:109B200025E007E04CF40006BE60A0F870200A2A89
:109B300001D22360F0BD142A01D22B60F0BDA0F841
:109B40007010F0BD2B60A0F8701080F86F10F0BDA1
:109B5000642E04D2A0F87020322AEED3E9E7A0F8F0
:109B60007010EAE77F1C80F86F70A0F8701090F812
:109B70006F20012A10D0002AE9D0B0F87060761C5E
:109B8000B6B2A0F870601E2ED7D323603C2EDED96B
:109B9000521E80F86F20D2E7B0F87020521C92B2AB
:109BA000A0F870202360C82AD1D980F86F10C6E7CA
:109BB000E805002048070020580E0020A4020020DD
:109BC000000C002038010020D0040020141C0140AB
:109BD000F0B54548B0F84810491C89B2A0F84810C3
:109BE00002297DD341490024A0F848400A78404B1F
:109BF000042A5BD04FF48041082A0BD0A0F10C025C
:109C0000B2F900208A4200DA1146B3F984208A4270
:109C100000DA1146374A12698A4200DA11B24182EB
:109C200082881D8AC2EB8502334D12B22D78C5F3AE
:109C300081062D4D40F6D9467243B5F97650921201
:109C40006A431213C26086681546C6EBC60642F325
:109C5000D102F60202EBA6328260C66C1644C664DC
:109C6000B0F850707F1CBFB2A0F85070B7F5806F8D
:109C700004D3B6120682A0F85040C464C66A891A9A
:109C8000A6EB461740F2545207EB07174A43A7EBDF
:109C9000C61602EB4602466A32444262B3F93430D9
:109CA000B2EB034F06DD1A04426206E01349B1F934
:109CB0000410AFE7002A00DA4462C162104990F84C
:109CC0003D2091F838108A420DD080F83D10B0F850
:109CD0004210A0F84410B0F84010A0F8421000E084
:109CE00001E0A0F84050F0BD380500203F070020FB
:109CF000A4020020F80D0020D00400200C0E00204B
:109D00003801002015481649B0F85A200B889A1AD5
:109D100092B20F2A20D30988A0F85A10B0F9001087
:109D20004FF48042C1EBC12141F35131A0F86C10D6
:109D30000C490B78A0F10C01022B06D1B1F90030CF
:109D4000934202DA1B1D0B8000E00A800021A0F87C
:109D5000601020F85C1F428070470000380500202A
:109D6000480700203F0700204FF6FF7202EA8002FA
:109D700010F4404315480ED0B3F5804F14D0B3F51E
:109D8000004F4FEA122216D0C2F5807330F813301C
:109D90005B424B8005E0120A30F812304B80C2F56E
:109DA000807230F812000FE0120AC2F5807330F8AA
:109DB00013304B8005E030F81230C2F580725B4200
:109DC0004B8030F81200404208807047F4B1000820
:109DD000104A518AD08A928A16384639A2F1110265
:109DE00000D54942002A00DA52421144002800DA24
:109DF00040420844084943F6284300B2B1F93620EE
:109E00005A43921340F2D733584302EBA030C8862E
:109E100070470000A402002038050020F0B59049EA
:109E200090480A8903889A1A92B23E2A1ED3008863
:109E3000088101F138004FF4FA63428A9A4202D253
:109E4000521C428200E04382874A92F82220802AF4
:109E50000CD302F03F020A70B1F90620402A06DB5B
:109E6000FF2A04D0C2883AB1521EC280F0BDBDE8BC
:109E7000F0407B48FFF75CBD428A9A42F6D30778F0
:109E80004FF0010E3A074FF0FF055BD5847A40F2A0
:109E9000DC52630708D444F004038372C28081F863
:109EA0000BE081F80AE04CE04378072B05D0032B48
:109EB00003D0052B01D0062B07D1660605D444F04C
:109EC00040038372C280052239E0654A5FEA437C21
:109ED00002F138024FF42076127A0DD55FEAC26C97
:109EE0000AD45FEA446C07D442F0100202723A06C8
:109EF00028D4C680192222E0DF0709D0970707D4AB
:109F0000670605D442F002020272C680042216E0FF
:109F10009F0709D5170707D4670605D442F0080242
:109F20000272C68003220AE01B070BD5530709D42F
:109F3000630607D442F004020272C6800B22CA7282
:109F40008A72CD80494AB2F92230B2F91A7003F20E
:109F50003D140022A74200DB0276414E444C06F13C
:109F60003806A479B6895FEAC46C06F101064FF49D
:109F7000C874B6B213D58681B6F57A7F05D9017A51
:109F800021F0800101728281F0BD037A1E06FBD4AC
:109F9000828143F080020272C480112035E09F422A
:109FA00016DA037E052B13D28681B6F5487F04D9D5
:109FB0008281027A22F040020272027A5606E3D4CB
:109FC0005B1C037642F040020272C48002201CE057
:109FD000284B1C89C4F3C006C4F3002740F2EE24CA
:109FE000BE4216D11E78360713D4427E012ACBD149
:109FF000428BB2F5167F02D2521C4283F0BD827AA8
:10A0000042F002028272C4800F20C8728872CD8032
:10A01000F0BD93F811714FF40046012F18D1164F7F
:10A0200041F6583C7F6C674512DD83F810E1134B15
:10A030001E60C38AA34202D25B1CC382F0BD4FF4F0
:10A04000FA73C3801C23CB728B72CD80C282F0BDA9
:10A05000C2820A4883F81021001F0660F0BD00008C
:10A06000D806002048070020E8050020D004002082
:10A07000000C0020A4020020380100201408014038
:10A080002DE9F05FDFF8FCB3FF489BF81830011DA5
:10A090000A1DFE4C012B5FD0B4F85E300380B4F88B
:10A0A00060000880B4F862001080FDF72FFBDFF835
:10A0B000E083F84D49F2CD32B8F91E00A883B8F913
:10A0C000201043F6CC4C00EB410151430914E983C5
:10A0D000B5F92230B5F9206001FB03F200FB06223E
:10A0E00042F38F326A82B5F91870714307FB0CF79F
:10A0F00040F2333CBF1302FB0CF207EBA23200FB31
:10A1000013102A8340F38F30A882B5F91A1043F652
:10A11000AE72514300EB0012891302EB8010DE4F48
:10A1200001EBA030DD4E6883786C306031693046D9
:10A130008847DB49308948800846FDF7C9FBD94E7E
:10A140004FF000094FF0010A307808280DD0698FD0
:10A150002982042833D01BE0B4F864300380B4F8BB
:10A1600066000880B4F868009EE7CF4890F9371081
:10A17000491C022921D890F8741019B1B5F85A0079
:10A18000288205E0698F2982A5F85A1080F874A00A
:10A19000B5F91410B5F90A00C44AF8F759FBE8629A
:10A1A000B4F91A11884204DDC048E962027C91408A
:10A1B00081623078042816D00CE0688FE0E7D8F888
:10A1C00024000014E862E07B04280CD0C5F82C9031
:10A1D00086F80090B54AB5F91210B5F90800303A82
:10A1E000F8F736FB02E0B87AF0B3B148A862A94D9F
:10A1F000AE4E443EA86A3060E86A70603046103562
:10A20000FBF762FD2888A5F14C01FFF7ADFDA5F134
:10A210005C08D8F81010C8F86C10B5F91020B068B8
:10A22000B5F9121000FB02F7F368484303FB1176FF
:10A2300046F38F3703FB0200AF8740F38F36EE877C
:10A240009C4D28466F80AE80FDF784FF287F08F183
:10A250001405012833D0704242104DF6B3504743E5
:10A260006A803914298000E026E04046A8F80060A2
:10A2700053184380511AA8F8041084F80C90B8F9C8
:10A280000030002B01DD84F80CA0B8F90200002892
:10A2900002DD217B891C2173B8F90420002A02DD2C
:10A2A000217B091D2173217B072920D2DFE801F0E2
:10A2B0001F1B3418301D32004FF4AF7096E77D48F5
:10A2C000B0F9203059424A106A80B0F91E004DF6AC
:10A2D000B3514843011429804046A8F80030C7E72D
:10A2E00084F80DA003E0022100E003216173DFF890
:10A2F000A4A1714E714F9AF800100129617B0DD015
:10A30000072972D2DFE801F071FCFBFAF9F8F700D7
:10A310000421EBE70521E9E70621E7E70729F0D269
:10A32000DFE801F063042F6489D5EF000146184689
:10A33000FBF74EFA2860B5F9020040F68151484318
:10A3400081136980B5F9000040F6815250438013B3
:10A3500028800A18A2F68152B8F80A305242C3EB9C
:10A36000620212B2A8F80820002A01DCA8F80890BE
:10A37000B8F80820A4F862201144A4F8601008443A
:10A380006DE1404201B2504200B2FBF721FA286071
:10A39000B5F9020040F68151484381136980B5F94F
:10A3A000000040F681525043801328800A18A2F61C
:10A3B0008152B8F80A305242C3EB620212B2A8F8D6
:10A3C0000820002A01DCA8F80890B8F80820A4F8B2
:10A3D00062201144A4F85E1008446EE13046F6F79E
:10A3E0004DFC01231A460721CAE0D4E01946104665
:10A3F000FBF7EEF92860B5F9020040F681514843B9
:10A4000080136880B5F9001040F6815251438913DA
:10A4100029804218A2F68152B8F80A305242C3EBA2
:10A42000620212B2A8F80820002A01DCA8F80890FD
:10A43000B8F8082068E15942404209B200B2FBF77F
:10A44000C7F92860B5F9020040F6815148438013EE
:10A450006880B5F9001040F6815251438913298074
:10A460004218A2F68152B8F80A305242C3EB620297
:10A4700012B2A8F80820002A01DCA8F80890B8F861
:10A48000082071E13C0B0020342C0140A402002084
:10A49000380500204C000020380100204004002036
:10A4A000FC0300203F070020140C0020000A0020BD
:10A4B000A2FEFFFF700B0020002401400028014095
:10A4C0003046F6F7DBFB01231A46052158E011461A
:10A4D000FBF77EF92860B5F9020040F68151484348
:10A4E00080136880B5F9001040F6815251438913FA
:10A4F0002980421806E076E14AE11BE1ECE0BCE08D
:10A500008FE010E0A2F68152B8F80A305242C3EB55
:10A51000620212B2A8F80820002A01DCA8F808900C
:10A52000B8F808204BE1504201B2584200B2FBF7A4
:10A530004FF92860B5F9020040F681514843801375
:10A540006880B5F9001040F6815251438913298083
:10A550004218A2F68152B8F80A305242C3EB6202A6
:10A5600012B2A8F80820002A01DCA8F80890B8F870
:10A57000082052E13046F6F781FB01231A460621F6
:10A580003846F6F77BFB01213046F6F7EDFA01215C
:10A590003846F6F7E9FABAF80800ABF80000BAF85E
:10A5A0000A00ABF80200BAF81000ABF804005546F8
:10A5B0005E46AB48F8F70AFBB4F85E00F188084441
:10A5C000A4F86400B4F8600031890844A4F8660077
:10A5D000B4F8620071890844A4F86800317EA1488B
:10A5E000012978D034F85E1F018061884180A188FC
:10A5F00081809C49028808310A8042884A8080888C
:10A6000088809848896A0830884795F83E00002875
:10A610007ED0F7F725FF15F83E0F401E2870BDE8E5
:10A62000F09F01461846FBF7D3F82860B5F9020001
:10A6300040F68151484380136880B5F9001040F618
:10A640008152514389134218A2F681525242520854
:10A650002980A4F862201044A4F860000844A4F8FB
:10A660005E0000213046F6F77FFA00213846F6F703
:10A670007BFA01231A460621B0E6404201B250425D
:10A6800000B2FBF7A5F82860B5F9020040F6815149
:10A69000484380136880B5F9001040F68152514359
:10A6A00089134218A2F68152524252082980A4F816
:10A6B00062201044A4F85E000844A4F86000002161
:10A6C0003046F6F751FA00213846F6F74DFA0123E5
:10A6D0001A46052182E6B4E019461046FBF778F8E1
:10A6E0002860B5F9020040F6815148438013688024
:10A6F000B5F9001040F68152514389134218A2F671
:10A700008152524229805208A4F85E20104400E091
:10A710009AE0A4F862000844A4F8600000213046E2
:10A72000F6F722FA00213846F6F71EFA01231A46F8
:10A730000721C5E65942404209B200B2FBF748F88A
:10A740002860B5F9020040F68151484380136880C3
:10A75000B5F9001040F68152514389134218A2F610
:10A760008152524229805208A4F85E201044A4F875
:10A7700060000844A4F8620000213046F6F7F4F9BE
:10A7800000213846F6F7F0F901231A46062197E62C
:10A790001146FBF71DF82860B5F9020040F681511B
:10A7A000484380136880B5F9001040F68152514348
:10A7B00089134218A2F68152524229805208A4F805
:10A7C00060201044A4F85E000844A4F86200002150
:10A7D0003046F6F7C9F900213846F6F7C5F90123E6
:10A7E0001A460521C6E6504201B2584200B2FAF7B5
:10A7F000EFFF2860B5F9020040F68151484380130D
:10A800006880B5F9001040F681525143891342180F
:10A81000A2F68152524229805208A4F860201044C6
:10A82000A4F862000844A4F85E0000213046F6F760
:10A830009BF900213846F6F797F901231A460721BC
:10A8400098E634F8641FCFE607480088A0F5D041A9
:10A8500068393FF4E4AEBDE8F05FF8F765BC00008E
:10A860003C0B002018000020182C01402DE9F0417D
:10A87000944C9548B4F862100288511A89B20F2995
:10A880006FD30088A4F8620090480088DFF8408207
:10A89000C0074FF000054FF0010741D08B4AD4E9C3
:10A8A0000C1024321388B1EB530F02D21288511AC4
:10A8B00008444FF4F371884200D208468549B1FB41
:10A8C000F0F0616CC1F35101084406466064F5F78D
:10A8D000B2FD0022804BF5F71AFD4FF040427F4B4E
:10A8E000F5F715FD0E22F5F781FDF5F7DBFDA4F870
:10A8F000AC0094F86D00401CC0B284F86D000828CC
:10A9000034D3704898F84A20001F03789A4201D047
:10A9100002704580724A1378724A23B1458021E063
:10A920006564256569E0D8F89810A1F5FA618E4252
:10A9300011DDE16D8B1C9E4205DDB0F902100A2984
:10A940000DDA491C06E08E4205DAB0F90210002942
:10A9500008DD491E4180B0F902000A2802DB1770A9
:10A9600001E0ABE01570E66584F86D505E484FF489
:10A97000A5420178C1F38101012962D044F25063FC
:10A98000A4F80830A4F8A820B0F9243021894B435A
:10A990009B13A4F8A430B0F90E00D4F850C0704353
:10A9A000B0FBF1F35149CCEBCC0C4FEACC2C09882D
:10A9B000C3F3D10303EB9C33B0032365B0FBF1F188
:10A9C0004B4BC908B3F846C0CCEBCC0C4FEACC2CAF
:10A9D00001EB9C31A3F84610F117890341EA964137
:10A9E0000023F5F79FFBB4F8AA10C1EBC101C9021F
:10A9F000C00800EB9130A4F8AA00616C206F0844F5
:10AA0000206794F87420521CD2B284F87420082A6B
:10AA100005D3C008A4F8760084F87450256735483B
:10AA2000C3885A0605D498F80F20022A0DD0A4F83E
:10AA30008A50244894F83F20B8300C2A28D2C57494
:10AA400027E045F6C05121819CE794F8382094F81E
:10AA50008E60B2420CD084F88E2094F83D2002F033
:10AA60000106C2F34002964202D1A4F88A5005E0E2
:10AA7000B4F88A2040F6B836B24205D2B4F88A005B
:10AA8000401CA4F88A00D4E743F08002C280D0E7DB
:10AA9000C774194B0E4C41F2482693F83C30B4F879
:10AAA000864041F2504C0C2A0AD3B14208DB012BFC
:10AAB00006D0614502DD002C00D18774BDE8F0812D
:10AAC0008574FBE73801002048070020000400409F
:10AAD000A40200204564BD0100209C40133B33408C
:10AAE000FA030020FB030020D004002030010020E6
:10AAF000300A0020000C00203805002070B5394CC9
:10AB0000394821880288511A89B23E294DD30088DC
:10AB1000364E20803649307806F1140518B3488B3C
:10AB200080002880E96828468847B5F90400314943
:10AB3000FCF79FFD304A60804FF48045D3884FF08A
:10AB400000015E0737D4B0F5DC5F2FDDE079401CF3
:10AB5000C0B2E0710A283ED343F4004040F0040044
:10AB6000D080A16036E0888B204A8000121D1080C2
:10AB7000888B80005080888B800000B290804A8B48
:10AB800092002A804A8B92006A80498B8900A980B2
:10AB900018497C31FCF76DFDA080B5F9040015491A
:10ABA000FCF767FD60800120307070BD23F4004029
:10ABB000A560D0800EE043F4004343F00403A1609D
:10ABC000D380B0F5B45F06DC23F4004020F004002D
:10ABD000D080A560E171D4E90201884200DB08461B
:10ABE000206170BDF80D0020480700209406002069
:10ABF000A4020020ECB70008000C002005494FF427
:10AC00008040C860886008610348C18821F482716F
:10AC1000C1807047F80D0020000C00202DE9F041A4
:10AC2000384C394E394F207841F23331C2074FF05A
:10AC300000050CD0A28962B394F90700002800DA5D
:10AC40004042C0B2032829D240F2AE702AE0A5707B
:10AC5000E5732F4AE571A58192F83830237220F010
:10AC60000800A18040F002002070BD867560B560CC
:10AC7000F560116D490005D041F68461A18140F075
:10AC800010002070C0B240F0010020706574BDE873
:10AC9000F081658120F01000207015E0042803D2B7
:10ACA00040F6510060810FE0052802D240F699106D
:10ACB000F8E740F6CC42062803D3072801D308283A
:10ACC00001D2628100E0618197F8A10098B9B08853
:10ACD000102301B2B4F90A003622FBF737FD706089
:10ACE000F168401AB1680844B060B6F900104843F2
:10ACF000C013F060B886B88E10B10120A070C6E70E
:10AD0000A570C4E70C0E0020B8060020A4020020A5
:10AD1000380100202DE9F041554C2678F0077CD011
:10AD20005448217A544D90F8380081427BD0534AE0
:10AD30002346DFF84CC1575C93F90E2093F9073096
:10AD4000874203D01CF80170874213D146F00206F7
:10AD50005B1C26705BB2E3711CF80110814201D1CB
:10AD60005B1CE37194F90710062901DD0621E171EE
:10AD7000521C1CE0434F17F801C0434F844503D0D9
:10AD800017F801C0844513D126F002065B1E267019
:10AD90005BB2E371795C814201D15B1EE37194F98E
:10ADA00007306FF005018B4200DAE171521EA27389
:10ADB000207294F907108A1C042A02D941F6846291
:10ADC000A2812C4A012912780ADD2B4B56079B6879
:10ADD00002D543F0080301E023F00803AB60607084
:10ADE000B1F1FF3F09DA5107A96802D521F0080146
:10ADF00001E041F00801A9606070F8F7CFFCA0788D
:10AE0000012810D121488068A3280CDA94F90700A2
:10AE1000022803DD0220E07105E01EE06FF0010171
:10AE2000884200DAE171A089002630B1401E00049A
:10AE3000000CA08101D1E671A673E87B04280CD038
:10AE4000B5F93410512341220020FBF77FFCA8867E
:10AE5000002802D1E07B10B1A670BDE8F0810C485B
:10AE600006700C480670207820F001002070F4E78E
:10AE70000C0E002038010020A4020020E4B80008D5
:10AE8000EAB80008F6B80008FCB800083805002049
:10AE90005C0700203F070020F0B415460D4A0E461F
:10AEA0004FF0FF31B0EBA20F12DA002810DB0A4995
:10AEB000096851F82000406844682CB129463046A2
:10AEC000A446F0BC1A4660476FF00500F0BC70471E
:10AED0000846FBE7040000007C080020173E573CB2
:10AEE000BB3A3E39DD379436613541343333353240
:10AEF000443161308A2FBD2EFB2D412DCC1C58587A
:10AF000058689919585858683313005695130054C7
:10AF1000B61300525A140050FD14004EA115004CF7
:10AF20004516004A761600486C1700467218004411
:10AF3000BA190042741B0040911D003EB420003C31
:10AF40009F22003AE1220038532300368B2400343C
:10AF5000812500322B2700302028002E5829002C74
:10AF6000B02A002A9B2C0028D22D00267C2F0024FA
:10AF70002631002202330020FD34001E5C37001C05
:10AF8000CC3C001A873E0018BE3F0016004000145B
:10AF900000400012004000100040000E0040000C75
:10AFA0000040000A00400008004000060040000485
:10AFB00000400002004000000102030405000500FB
:10AFC000010203040104000305020000F001000077
:10AFD00036010000F8000000BA0000007C0000000C
:10AFE0007C0000007C000000C91C9C19991CCC1935
:10AFF0009C1CC9190000290052007B00A400CC0051
:10B00000F5001E01470170019901C201EA01130216
:10B010003C0265028E02B602DF02080330035903C8
:10B020008203AA03D303FB0324044C0475049D0488
:10B03000C504EE0416053E0567058F05B705DF0557
:10B0400007062F0657067F06A706CE06F6061E073A
:10B0500046076D079507BC07E4070B083208590837
:10B060008108A808CF08F6081D0944096A09910952
:10B07000B809DE09050A2B0A520A780A9E0AC40A90
:10B08000EA0A100B360B5C0B820BA80BCD0BF30BF3
:10B09000180C3E0C630C880CAD0CD20CF70C1C0D7C
:10B0A000410D650D8A0DAF0DD30DF70D1C0E400E31
:10B0B000640E880EAC0ECF0EF30E170F3A0F5E0F14
:10B0C000810FA40FC70FEA0F0D1030105310751029
:10B0D0009810BA10DD10FF1021114311651187116E
:10B0E000A911CA11EC110D122E12501271129212E6
:10B0F000B312D412F4121513361356137613961393
:10B10000B713D713F6131614361456147514941473
:10B11000B414D314F214111530154E156D158C1589
:10B12000AA15C815E7150516231641165F167C16D5
:10B130009A16B716D516F2160F172C174917661759
:10B140008317A017BC17D917F51711182E184A180E
:10B15000661881189D18B918D418F0180B192619FB
:10B1600042195D1978199219AD19C819E219FD191A
:10B17000171A311A4C1A661A801A991AB31ACD1A6C
:10B18000E61A001B191B331B4C1B651B7E1B971BF0
:10B19000AF1BC81BE11BF91B121C2A1C421C5A1CAA
:10B1A000721C8A1CA21CBA1CD21CE91C011D181D91
:10B1B000301D471D5E1D751D8C1DA31DBA1DD01DA4
:10B1C000E71DFD1D141E2A1E401E571E6D1E831EE8
:10B1D000981EAE1EC41EDA1EEF1E051F1A1F2F1F5B
:10B1E000451F5A1F6F1F841F991FAE1FC21FD71FF5
:10B1F000EC1F002000006400C9002D019201F7013E
:10B200005B02C00224038903ED035204B6041A054D
:10B210007F05E3054706AB060F077307D7073B0813
:10B220009F0802096609C9092D0A900AF30A560BFC
:10B23000B90B1C0C7F0CE20C440DA60D090E6B0E15
:10B24000CD0E2F0F900FF20F5310B4101511761171
:10B25000D71138129812F8125813B813181477141B
:10B26000D61435159415F3155116B0160E176B1725
:10B27000C91726188318E0183D199919F519511A9C
:10B28000AD1A081B631BBE1B181C731CCD1C261D8E
:10B29000801DD91D321E8A1EE31E3B1F921FEA1F0E
:10B2A00041209820EE2044219A21EF214522992225
:10B2B000EE2242239623E9233C248F24E2243425E2
:10B2C0008525D72528267826C82618276827B72752
:10B2D00006285428A228EF283D298929D629222A80
:10B2E0006D2AB82A032B4D2B972BE12B2A2C722C7D
:10B2F000BB2C022D4A2D912DD72D1D2E632EA82E4D
:10B30000EC2E302F742FB82FFA2F3D307F30C03005
:10B31000013141318131C13100323F327D32BA32A7
:10B32000F73234337033AC33E73322345C34953442
:10B33000CE3407353F357735AE35E4351A365036DD
:10B340008536B936ED36203753378637B737E93784
:10B35000193849387938A838D738053932395F393A
:10B360008B39B739E2390D3A373A603A893AB23A0D
:10B37000DA3A013B283B4E3B733B983BBD3BE03BFD
:10B38000043C263C483C6A3C8B3CAB3CCB3CEA3C16
:10B39000093D273D443D613D7D3D993DB43DCE3D58
:10B3A000E83D013E1A3E323E493E603E763E8C3ECE
:10B3B000A13EB53EC93EDC3EEF3E013F123F233F7A
:10B3C000333F433F513F603F6E3F7B3F873F933F5B
:10B3D0009E3FA93FB33FBC3FC53FCD3FD53FDC3F7C
:10B3E000E23FE83FED3FF13FF53FF93FFB3FFD3FD7
:10B3F000FF3FFF3FFF3F0000E0203420002020E01F
:10B400002020202337202620210000800200040075
:10B4100008001000000200040008040000020004FC
:10B4200000080010002000400080040000000080A0
:10B430000000004000000020000000100000000894
:10B440000000000400000002000000010000800075
:10B450000000400000002000000010000000080074
:10B460000000040000000200000001000080000055
:10B4700000080140000C0140000C0140000C01409C
:10B48000000C0140000C0140000C0140000C014088
:10B490000010014000100140001001400010014068
:10B4A0000010014000100140001001400010014058
:10B4B0000014014004080140040C0140040C014048
:10B4C000040C0140040C0140040C0140040C014038
:10B4D000040C01400410014004100140041001401C
:10B4E0000410014004100140041001400410014008
:10B4F000041001400414014008080140080C0140F8
:10B50000080C0140080C0140080C0140080C0140E7
:10B51000080C0140080C01400810014008100140CF
:10B5200008100140081001400810014008100140B7
:10B530000810014008100140081401400C080140A7
:10B540000C0C01400C0C01400C0C01400C0C014097
:10B550000C0C01400C0C01400C0C01400C10014083
:10B560000C1001400C1001400C1001400C10014067
:10B570000C1001400C1001400C1001400C14014053
:10B5800010080140100C0140100C0140100C01404B
:10B59000100C0140100C0140100C0140100C014037
:10B5A0001010014010100140101001401010014017
:10B5B0001010014010100140101001401010014007
:10B5C0001014014000000000000000000000000016
:10B5D000000000000000000014080140140C0140AD
:10B5E000140C0140140C0140140C0140140C0140D7
:10B5F000140C0140140C01401410014014100140BF
:10B6000014100140141001401410014014100140A6
:10B6100014100140141001401414014000000000F7
:10B62000000000000000000000000000000000001A
:10B63000FFFFFF0F0FFFFFFFFFF0FFFFFF0FFFFFF9
:10B64000FFFFF0FF0FFFFFFFFFF0FFFFFF0FFFFF08
:10B65000FFF0FFFF0FFFFFFFFFF0FFFFFF0FFFFFF8
:10B66000FFFFF0FFFFFF0FFFFFFFFFF0FFFFFF0FE8
:10B67000FFF0FFFF00000040400000000004000059
:10B680000040000000000400400000000004000032
:10B690000040000000040000400000000004000022
:10B6A0000040000000000400000040000000000412
:10B6B0000000004000040000000000808000000046
:10B6C000000800000080000000000800800000006A
:10B6D000000800000080000000080000800000005A
:10B6E000000800000080000000000800000080004A
:10B6F000000000080000008000080000000000209A
:10B7000020000000000200000020000000000200F5
:10B7100020000000000200000020000000020000E5
:10B7200020000000000200000020000000000200D5
:10B7300000002000000000020000002000020000C5
:10B7400000000060600000000006000000600000D3
:10B75000000006006000000000060000006000001D
:10B76000000600006000000000060000006000000D
:10B7700000000600000060000000000600000060FD
:10B780000006000000800200040008001000000213
:10B79000000400080400000200040008001000205B
:10B7A0000040008004000000FF7FFFFFFDFFFFFF5F
:10B7B000FBFFFFFFF7FFFFFFEFFFFFFFFFFDFFFFB7
:10B7C000FFFBFFFFFFF7FFFFFBFFFFFFFFFDFFFF9B
:10B7D000FFFBFFFFFFF7FFFFFFEFFFFFFFDFFFFFB5
:10B7E000FFBFFFFFFF7FFFFFFBFFFFFF401FFC02CC
:10B7F000001E5A03C01CC403801B3C04401AC6042C
:10B8000000196305C01717068016E4064015CD071A
:10B810000014D708C012050A80115B0B4010DD0C24
:10B82000000F900EC00D7510800C9012400BE014AC
:10B83000000A6517C0081C1A8007FD1C400600207E
:10B8400000051823C003372680024E2940014C2CE6
:10B850000000242FC0FEC73180FD2E3400FB2D38A0
:10B8600080F81C3B00F6003C8025151A40249A1BEA
:10B8700000231E1DC021B81E80205D20401F0C2209
:10B88000001EC223C01C7E25801B3327401AFB28C4
:10B890000019B72AC0176D2C8016192E4015B92F24
:10B8A00000144731C012C9328011353440108B3535
:10B8B000000FCA36C00DF037800CFE38400BF4394B
:10B8C000000AD23AC008983B8007473C4006E13C5A
:10B8D0000005673DC003DA3D80023E3E4001923ED6
:10B8E0000000143F010203040500020304050001E7
:10B8F0000304050001020500010203040405000120
:10B90000020355050010AA1A55250030AA3A000076
:10B91000AA0A55150020AA2A5535FF3F6465765FAF
:10B9200063616E3100000000298A0008D98B00088D
:10B93000558B0008858900084D890008000000002B
:10B940001CB9000828B900086CB9000800000020E4
:10B950008C0800000007000898BA00088C08002036
:10B960003C1500008085000840B9000801441371AF
:10B97000401B088504211355152A4006190801A704
:10B9800013CB5A1B08F1041AEB04012423286E423E
:10B990000117020604050103148020FF8BAA0A0286
:10B9A00001A415AA0A551500085920AA2A5535FFE1
:10B9B0003F073103010504060203127C1573FFFFE4
:10B9C00004FF808001012D025F6402130A13818C41
:10B9D00052081201100C05040602030101030705B9
:10B9E00005280B010203040206070303040C3D07AC
:10B9F00006040509191F191904310506060B14AAB6
:10BA00001A02312E40FD3969260211042F405F02CF
:10BA10000C26405B262ACD55155515123902017F9B
:10BA20000316D0071AFF01013B0261AA0C1008019E
:10BA300008A834993F33138194391CA9100916E8DA
:10BA400091220312100A17401C12600A16901B0163
:10BA50001AA2646B958C94012199D0019A5A140210
:10BA60001AC802CBD007023A19164902892612C811
:10BA7000DA01DA1AFF01C1227D130D0212103AFA1F
:10BA80000812081CF401010812062BE80310120228
:08BA90001B68B915B1000000AC
:020000040800F2
:10FC00004A46545A594D46312D4E3330202020203B
:10FC1000050406020301AA0AAA0AAA0AAA0AAA0A4B
:10FC2000AA0ADE3F00100000FF0131000301664612
:10FC300000400040513800400040004000400101B9
:10FC4000004000407A3B082708270827FF0033338D
:10FC50000201401F00016626B81E6626FFFFFFFF57
:10FC6000FFFF01010100010000000300000202008B
:04FC70000000AA5591
:04000005080000ED02
:00000001FF
